Archive member included because of file (symbol)

lib_generic/libgeneric.a(vsprintf.o)
                              cpu/mpc85xx/traps.o (panic)
lib_generic/libgeneric.a(ctype.o)
                              lib_generic/libgeneric.a(vsprintf.o) (_ctype)
lib_generic/libgeneric.a(string.o)
                              lib_generic/libgeneric.a(vsprintf.o) (strnlen)
board/mpc8548pc/libmpc8548pc.a(mpc8548pc.o)
                              cpu/mpc85xx/speed.o (get_clock_freq)
lib_ppc/libppc.a(ppcstring.o)
                              lib_generic/libgeneric.a(string.o) (strcpy)
lib_ppc/libppc.a(board.o)     common/dlmalloc.o (sbrk)
lib_ppc/libppc.a(time.o)      lib_generic/libgeneric.a(vsprintf.o) (udelay)
lib_ppc/libppc.a(ticks.o)     lib_ppc/libppc.a(time.o) (wait_ticks)
net/libnet.a(net.o)           lib_ppc/libppc.a(board.o) (copy_filename)
net/libnet.a(tftp.o)          net/libnet.a(net.o) (TftpStart)
net/libnet.a(bootp.o)         net/libnet.a(net.o) (BootpTry)
net/libnet.a(rarp.o)          net/libnet.a(net.o) (RarpTry)
net/libnet.a(eth.o)           net/libnet.a(net.o) (eth_get_dev)
net/libnet.a(nfs.o)           net/libnet.a(net.o) (NfsStart)
drivers/libdrivers.a(cfi_flash.o)
                              lib_ppc/libppc.a(board.o) (flash_init)
drivers/libdrivers.a(pci.o)   cpu/mpc85xx/pci.o (pci_register_hose)
drivers/libdrivers.a(pci_auto.o)
                              drivers/libdrivers.a(pci.o) (pciauto_config_init)
drivers/libdrivers.a(pci_indirect.o)
                              cpu/mpc85xx/pci.o (pci_setup_indirect)
drivers/libdrivers.a(serial.o)
                              lib_ppc/libppc.a(board.o) (serial_init)
drivers/libdrivers.a(tsec.o)  board/mpc8548pc/libmpc8548pc.a(mpc8548pc.o) (tsec_miiphy_write)
drivers/libdrivers.a(ns16550.o)
                              drivers/libdrivers.a(serial.o) (NS16550_init)
common/libcommon.a(main.o)    lib_ppc/libppc.a(board.o) (main_loop)
common/libcommon.a(cmd_autoscript.o)
                              (__u_boot_cmd_autoscr)
common/libcommon.a(cmd_bdinfo.o)
                              (__u_boot_cmd_bdinfo)
common/libcommon.a(cmd_boot.o)
                              (__u_boot_cmd_reset)
common/libcommon.a(cmd_bootm.o)
                              (__u_boot_cmd_imls)
common/libcommon.a(cmd_console.o)
                              (__u_boot_cmd_coninfo)
common/libcommon.a(cmd_flash.o)
                              (__u_boot_cmd_protect)
common/libcommon.a(cmd_i2c.o)
                              (__u_boot_cmd_iloop)
common/libcommon.a(cmd_itest.o)
                              (__u_boot_cmd_itest)
common/libcommon.a(cmd_load.o)
                              (__u_boot_cmd_loadb)
common/libcommon.a(cmd_mem.o)
                              (__u_boot_cmd_mtest)
common/libcommon.a(cmd_mii.o)
                              (__u_boot_cmd_mii)
common/libcommon.a(cmd_misc.o)
                              (__u_boot_cmd_sleep)
common/libcommon.a(cmd_net.o)
                              (__u_boot_cmd_ping)
common/libcommon.a(cmd_nvedit.o)
                              (__u_boot_cmd_run)
common/libcommon.a(cmd_pci.o)
                              (__u_boot_cmd_pci)
common/libcommon.a(command.o)
                              (__u_boot_cmd_question_mark)
common/libcommon.a(console.o)
                              cpu/mpc85xx/traps.o (printf)
common/libcommon.a(devices.o)
                              common/libcommon.a(cmd_console.o) (stdio_names)
common/libcommon.a(env_common.o)
                              common/libcommon.a(cmd_nvedit.o) (env_get_char)
common/libcommon.a(env_flash.o)
                              common/libcommon.a(env_common.o) (env_ptr)
common/libcommon.a(exports.o)
                              lib_ppc/libppc.a(board.o) (jumptable_init)
common/libcommon.a(flash.o)   drivers/libdrivers.a(cfi_flash.o) (flash_protect)
common/libcommon.a(hush.o)    common/libcommon.a(main.o) (u_boot_hush_start)
common/libcommon.a(lists.o)   common/libcommon.a(devices.o) (ListCreate)
common/libcommon.a(miiphyutil.o)
                              net/libnet.a(eth.o) (miiphy_init)
common/libcommon.a(s_record.o)
                              common/libcommon.a(cmd_load.o) (srec_decode)
lib_generic/libgeneric.a(display_options.o)
                              lib_ppc/libppc.a(board.o) (display_options)
cpu/mpc85xx/libmpc85xx.a(i2c.o)
                              lib_ppc/libppc.a(board.o) (i2c_init)
lib_ppc/libppc.a(cache.o)     common/libcommon.a(cmd_load.o) (flush_cache)

Allocating common symbols
Common symbol       size              file

dp_last_size        0x4               common/libcommon.a(cmd_mem.o)
console_buffer      0x100             common/libcommon.a(main.o)
NetArpWaitTry       0x4               net/libnet.a(net.o)
NetArpWaitPacketMAC
                    0x4               net/libnet.a(net.o)
last_reg_hi         0x4               common/libcommon.a(cmd_mii.o)
flash_info          0x590             drivers/libdrivers.a(cfi_flash.o)
NetOurEther         0x6               net/libnet.a(net.o)
NetOurIP            0x4               net/libnet.a(net.o)
NetPingIP           0x4               net/libnet.a(net.o)
NetServerIP         0x4               net/libnet.a(net.o)
monitor_flash_len   0x4               lib_ppc/libppc.a(board.o)
___strtok           0x4               lib_generic/libgeneric.a(string.o)
NetArpWaitTxPacketSize
                    0x4               net/libnet.a(net.o)
NetArpWaitReplyIP   0x4               net/libnet.a(net.o)
NetRxPackets        0x10              net/libnet.a(net.o)
NetArpWaitTxPacket  0x4               net/libnet.a(net.o)
NetArpWaitPacketIP  0x4               net/libnet.a(net.o)
NetState            0x4               net/libnet.a(net.o)
BootpTry            0x4               net/libnet.a(bootp.o)
BootFile            0x80              net/libnet.a(net.o)
dp_last_addr        0x4               common/libcommon.a(cmd_mem.o)
his_pad_char        0x1               common/libcommon.a(cmd_load.o)
last_data           0x4               common/libcommon.a(cmd_mii.o)
os_data_count       0x4               common/libcommon.a(cmd_load.o)
RarpTry             0x4               net/libnet.a(rarp.o)
last_addr_hi        0x4               common/libcommon.a(cmd_mii.o)
mm_last_size        0x4               common/libcommon.a(cmd_mem.o)
os_data_init        0x4               common/libcommon.a(cmd_load.o)
mm_last_addr        0x4               common/libcommon.a(cmd_mem.o)
NetIPID             0x4               net/libnet.a(net.o)
last_reg_lo         0x4               common/libcommon.a(cmd_mii.o)
nesting_level       0x4               common/libcommon.a(hush.o)
send_ptr            0x4               common/libcommon.a(cmd_load.o)
BootpID             0x4               net/libnet.a(bootp.o)
last_return_code    0x4               common/libcommon.a(hush.o)
NetRxPkt            0x4               net/libnet.a(net.o)
os_data_header      0x20              common/libcommon.a(cmd_load.o)
os_data_char        0x4               common/libcommon.a(cmd_load.o)
last_op             0x2               common/libcommon.a(cmd_mii.o)
NetArpWaitPacketBuf
                    0x620             net/libnet.a(net.o)
his_eol             0x1               common/libcommon.a(cmd_load.o)
header              0x40              common/libcommon.a(cmd_bootm.o)
NetRxPktLen         0x4               net/libnet.a(net.o)
his_quote           0x1               common/libcommon.a(cmd_load.o)
NetBootFileXferSize
                    0x4               net/libnet.a(net.o)
last_addr_lo        0x4               common/libcommon.a(cmd_mii.o)
PktBuf              0x1e20            net/libnet.a(net.o)
send_parms          0x14              common/libcommon.a(cmd_load.o)
his_pad_count       0x4               common/libcommon.a(cmd_load.o)
NetArpWaitTimerStart
                    0x4               net/libnet.a(net.o)
decrementer_count   0x4               cpu/mpc85xx/interrupts.o

Memory Configuration

Name             Origin             Length             Attributes
*default*        0x00000000         0xffffffff

Linker script and memory map


.resetvec       0xfffffffc        0x4
 *(.resetvec)
 .resetvec      0xfffffffc        0x4 cpu/mpc85xx/resetvec.o

.bootpg         0xfffff000      0x3d0
 cpu/mpc85xx/start.o(.bootpg)
 .bootpg        0xfffff000      0x258 cpu/mpc85xx/start.o
                0xfffff000                _start_e500
 board/mpc8548pc/init.o(.bootpg)
 .bootpg        0xfffff258      0x178 board/mpc8548pc/init.o
                0xfffff370                law_entry
                0xfffff258                tlb1_entry

.rela.dyn
                0x00000094                . = SIZEOF_HEADERS

.interp
 *(.interp)

.hash
 *(.hash)

.dynsym
 *(.dynsym)

.dynstr
 *(.dynstr)

.rel.text
 *(.rel.text)

.rela.text
 *(.rela.text)

.rel.data
 *(.rel.data)

.rela.data
 *(.rela.data)

.rel.rodata
 *(.rel.rodata)

.rela.rodata
 *(.rela.rodata)

.rel.got
 *(.rel.got)

.rela.got
 *(.rela.got)

.rel.ctors
 *(.rel.ctors)

.rela.ctors
 *(.rela.ctors)

.rel.dtors
 *(.rel.dtors)

.rela.dtors
 *(.rela.dtors)

.rel.bss
 *(.rel.bss)

.rela.bss
 *(.rela.bss)

.rel.plt
 *(.rel.plt)

.rela.plt
 *(.rela.plt)

.init
 *(.init)

.plt
 *(.plt)

.text           0xfff80000    0x1eb14
 cpu/mpc85xx/start.o(.text)
 .text          0xfff80000     0x2710 cpu/mpc85xx/start.o
                0xfff801e8                _start_of_vectors
                0xfff80004                version_string
                0xfff823dc                dcache_enable
                0xfff824d0                relocate_code
                0xfff824a0                in32
                0xfff82498                in16r
                0xfff826e0                unlock_ram_in_cache
                0xfff8243c                get_pir
                0xfff82460                in8
                0xfff824a8                in32r
                0xfff82470                out16
                0xfff82490                in16
                0xfff8238c                icache_enable
                0xfff82458                wr_tcr
                0xfff82100                transfer_to_handler
                0xfff824b8                ppcDcbi
                0xfff80100                _start
                0xfff824c8                ppcSync
                0xfff824c0                ppcDcbz
                0xfff82480                out32
                0xfff82444                get_pvr
                0xfff823b4                icache_disable
                0xfff82478                out16r
                0xfff82468                out8
                0xfff80f90                _end_of_vectors
                0xfff82430                dcache_status
                0xfff82488                out32r
                0xfff824b0                ppcDcbf
                0xfff8262c                trap_init
                0xfff823d0                icache_status
                0xfff8240c                dcache_disable
                0xfff8244c                get_svr
 board/mpc8548pc/init.o(.text)
 cpu/mpc85xx/traps.o(.text)
 .text          0xfff82710      0x520 cpu/mpc85xx/traps.o
                0xfff82934                CritcalInputException
                0xfff82c20                addr_probe
                0xfff827e4                show_regs
                0xfff82714                print_backtrace
                0xfff82b70                UnknownException
                0xfff82a6c                AlignmentException
                0xfff82abc                ProgramCheckException
                0xfff82b40                PITException
                0xfff828d0                _exception
                0xfff82974                MachineCheckException
                0xfff82bd0                DebugException
 cpu/mpc85xx/interrupts.o(.text)
 .text          0xfff82c30      0x224 cpu/mpc85xx/interrupts.o
                0xfff82e18                set_timer
                0xfff82d90                reset_timer
                0xfff82c70                interrupt_init
                0xfff82dd4                get_timer
                0xfff82d1c                irq_free_handler
                0xfff82d10                irq_install_handler
                0xfff82d2c                timer_interrupt
                0xfff82c4c                disable_interrupts
                0xfff82c30                enable_interrupts
 cpu/mpc85xx/cpu_init.o(.text)
 .text          0xfff82e54      0x1b4 cpu/mpc85xx/cpu_init.o
                0xfff82e54                cpu_init_f
                0xfff82ed4                cpu_init_r
 cpu/mpc85xx/cpu.o(.text)
 .text          0xfff83008      0x400 cpu/mpc85xx/cpu.o
                0xfff832d4                get_tbclk
                0xfff832b8                do_reset
                0xfff83304                dma_init
                0xfff83334                dma_check
                0xfff833a4                dma_xfer
                0xfff8300c                checkcpu
 cpu/mpc85xx/speed.o(.text)
 .text          0xfff83408      0x148 cpu/mpc85xx/speed.o
                0xfff834e8                get_clocks
                0xfff83528                get_bus_freq
                0xfff83408                get_sys_info
 cpu/mpc85xx/pci.o(.text)
 .text          0xfff83550      0x154 cpu/mpc85xx/pci.o
                0xfff83550                pci_mpc85xx_init
 common/dlmalloc.o(.text)
 .text          0xfff836a4     0x1288 common/dlmalloc.o
                0xfff83a6c                malloc
                0xfff846e0                pvalloc
                0xfff84710                calloc
                0xfff8483c                malloc_usable_size
                0xfff840dc                realloc
                0xfff83708                malloc_trim
                0xfff836a8                malloc_bin_reloc
                0xfff8488c                mallopt
                0xfff84584                memalign
                0xfff8481c                cfree
                0xfff846b8                valloc
                0xfff837fc                free
 lib_generic/crc32.o(.text)
 .text          0xfff8492c      0x150 lib_generic/crc32.o
                0xfff84930                crc32
 lib_ppc/extable.o(.text)
 .text          0xfff84a7c       0xcc lib_ppc/extable.o
                0xfff84a80                search_exception_table
 lib_generic/zlib.o(.text)
 .text          0xfff84b48     0x2bb0 lib_generic/zlib.o
                0xfff859f0                inflate
                0xfff84f54                inflateInit2
                0xfff8516c                inflateIncomp
                0xfff87580                adler32
                0xfff84d98                inflateReset
                0xfff84e04                inflateSync
                0xfff850dc                inflateInit
                0xfff84cd8                inflateEnd
 *(.text)
 .text          0xfff876f8      0xa40 lib_generic/libgeneric.a(vsprintf.o)
                0xfff87adc                vsprintf
                0xfff877f0                simple_strtol
                0xfff880b0                panic
                0xfff88054                sprintf
                0xfff876fc                simple_strtoul
 .text          0xfff88138      0x560 lib_generic/libgeneric.a(string.o)
                0xfff885e0                memscan
                0xfff8857c                strswab
                0xfff88320                strnlen
                0xfff882cc                strrchr
                0xfff8860c                strstr
                0xfff8824c                strncmp
                0xfff88468                strtok
                0xfff881f4                strncat
                0xfff88364                strdup
                0xfff8851c                strsep
                0xfff8813c                strnicmp
                0xfff883b8                strspn
                0xfff88298                strchr
                0xfff88418                strpbrk
 .text          0xfff88698      0xa60 board/mpc8548pc/libmpc8548pc.a(mpc8548pc.o)
                0xfff88720                get_prompt
                0xfff88e34                pci_init_board
                0xfff886ac                get_br0
                0xfff88d40                local_bus_init
                0xfff88844                board_early_init_f
                0xfff88e74                checkboard
                0xfff88698                get_clock_freq
                0xfff88cd0                initdram
                0xfff88904                reset_phy
                0xfff88898                board_early_init_r
                0xfff888f0                misc_init_r
                0xfff88b00                fixed_sdram
                0xfff886e4                get_br1
 .text          0xfff890f8      0x29c lib_ppc/libppc.a(ppcstring.o)
                0xfff890f8                strcpy
                0xfff89210                memmove
                0xfff89218                memcpy
                0xfff8913c                strcat
                0xfff8936c                memchr
                0xfff89114                strncpy
                0xfff89200                bcopy
                0xfff8933c                memcmp
                0xfff892b4                backwards_memcpy
                0xfff891a4                memset
                0xfff89168                strcmp
                0xfff8918c                strlen
 .text          0xfff89394      0x740 lib_ppc/libppc.a(board.o)
                0xfff8960c                hang
                0xfff8975c                board_init_r
                0xfff8940c                strmhz
                0xfff89398                sbrk
                0xfff8963c                board_init_f
 .text          0xfff89ad4       0xf8 lib_ppc/libppc.a(time.o)
                0xfff89ad4                usec2ticks
                0xfff89bb0                init_timebase
                0xfff89b58                udelay
                0xfff89b7c                ticks2usec
 .text          0xfff89bcc       0x44 lib_ppc/libppc.a(ticks.o)
                0xfff89be4                wait_ticks
                0xfff89bcc                get_ticks
 .text          0xfff89c10     0x15d4 net/libnet.a(net.o)
                0xfff8ac58                getenv_IPaddr
                0xfff8a588                NetCksumOk
                0xfff89e4c                NetSetTimeout
                0xfff8a620                copy_filename
                0xfff8a5bc                NetEthHdrSize
                0xfff8a68c                ip_to_string
                0xfff89ff0                ArpTimeoutCheck
                0xfff8a720                NetReceive
                0xfff8abc0                string_to_ip
                0xfff8a1f8                NetSendUDPPacket
                0xfff8a6e4                print_IPaddr
                0xfff89c14                NetSetEther
                0xfff8ad6c                NetLoop
                0xfff89cb4                ArpRequest
                0xfff8ac80                VLAN_to_string
                0xfff8ad44                getenv_VLAN
                0xfff8a0a8                NetCksum
                0xfff8a100                NetSetIP
                0xfff8acf8                string_to_VLAN
                0xfff89eec                NetStartAgain
                0xfff89eac                NetSetHandler
                0xfff8a368                PingSend
                0xfff8a088                NetSendPacket
 .text          0xfff8b1e4      0x6a0 net/libnet.a(tftp.o)
                0xfff8b67c                TftpStart
 .text          0xfff8b884      0x6a8 net/libnet.a(bootp.o)
                0xfff8bca4                BootpRequest
 .text          0xfff8bf2c      0x1f8 net/libnet.a(rarp.o)
                0xfff8bfb0                RarpRequest
 .text          0xfff8c124      0x934 net/libnet.a(eth.o)
                0xfff8c168                eth_get_dev_by_name
                0xfff8c844                eth_halt
                0xfff8c278                eth_register
                0xfff8c128                eth_get_dev
                0xfff8c6f4                eth_try_another
                0xfff8c600                eth_set_enetaddr
                0xfff8c340                eth_initialize
                0xfff8c978                eth_set_current
                0xfff8c914                eth_rx
                0xfff8c1f8                eth_get_dev_index
                0xfff8c7a4                eth_init
                0xfff8ca10                eth_get_name
                0xfff8c8a8                eth_send
 .text          0xfff8ca58      0xd28 net/libnet.a(nfs.o)
                0xfff8d540                NfsStart
 .text          0xfff8d780     0x14f8 drivers/libdrivers.a(cfi_flash.o)
                0xfff8e398                flash_get_size
                0xfff8d7c8                flash_read_ushort
                0xfff8e1b0                flash_erase
                0xfff8e71c                flash_init
                0xfff8d900                flash_print_info
                0xfff8d808                flash_read_long
                0xfff8d7a4                flash_read_uchar
                0xfff8d780                flash_make_addr
                0xfff8e9fc                write_buff
 .text          0xfff8ec78      0xd50 drivers/libdrivers.a(pci.o)
                0xfff8f7c0                pci_cfgfunc_config_device
                0xfff8f7fc                pci_hose_scan_bus
                0xfff8f3fc                pci_hose_phys_to_bus
                0xfff8f7f0                pci_cfgfunc_do_nothing
                0xfff8ecc8                pci_hose_read_config_dword
                0xfff8ed68                pci_hose_read_config_byte_via_dword
                0xfff8f578                pci_hose_config_device
                0xfff8f718                pci_find_config
                0xfff8ed18                pci_hose_write_config_word
                0xfff8f134                pci_read_config_dword
                0xfff8f4b8                pci_hose_bus_to_phys
                0xfff8ee18                pci_hose_write_config_byte_via_dword
                0xfff8edc0                pci_hose_read_config_word_via_dword
                0xfff8f9a8                pci_init
                0xfff8f19c                pci_read_config_word
                0xfff8f970                pci_hose_scan
                0xfff8f3ac                pci_find_device
                0xfff8eeb0                pci_hose_write_config_word_via_dword
                0xfff8f270                pci_find_devices
                0xfff8ef50                pci_register_hose
                0xfff8efac                pci_bus_to_hose
                0xfff8ed40                pci_hose_write_config_dword
                0xfff8f0d8                pci_write_config_byte
                0xfff8eca0                pci_hose_read_config_word
                0xfff8f204                pci_read_config_byte
                0xfff8ecf0                pci_hose_write_config_byte
                0xfff8f07c                pci_write_config_word
                0xfff8f020                pci_write_config_dword
                0xfff8ec78                pci_hose_read_config_byte
 .text          0xfff8f9c8      0x5b4 drivers/libdrivers.a(pci_auto.o)
                0xfff8f9c8                pciauto_region_init
                0xfff8fbe4                pciauto_config_init
                0xfff8fa00                pciauto_region_allocate
                0xfff8fa60                pciauto_setup_device
                0xfff8f9dc                pciauto_region_align
                0xfff8fcb4                pciauto_config_device
 .text          0xfff8ff7c      0x1cc drivers/libdrivers.a(pci_indirect.o)
                0xfff900dc                pci_setup_indirect
 .text          0xfff90148      0x374 drivers/libdrivers.a(serial.o)
                0xfff90390                _serial_setbrg
                0xfff90408                serial_putc_raw
                0xfff90498                serial_setbrg
                0xfff90344                _serial_tstc
                0xfff90474                serial_tstc
                0xfff903e4                serial_putc
                0xfff902ac                _serial_puts
                0xfff9025c                _serial_putc_raw
                0xfff9017c                serial_init
                0xfff9042c                serial_puts
                0xfff902f8                _serial_getc
                0xfff90450                serial_getc
                0xfff901e4                _serial_putc
 .text          0xfff904bc     0x1040 drivers/libdrivers.a(tsec.o)
                0xfff908d8                mii_parse_cis8201
                0xfff913a0                get_priv_for_phy
                0xfff90928                mii_parse_dm9161_scsr
                0xfff909bc                mii_cis8204_setmode
                0xfff91408                tsec_miiphy_read
                0xfff91314                mii_parse_lxt971_sr2
                0xfff904bc                write_phy_reg
                0xfff9054c                phy_run_commands
                0xfff90504                read_phy_reg
                0xfff9069c                mii_parse_sr
                0xfff909e0                get_phy_info
                0xfff9067c                mii_cr_init
                0xfff908a0                mii_parse_rtl8201cp_sr
                0xfff90960                mii_cis8204_fixled
                0xfff90af0                tsec_initialize
                0xfff91484                tsec_miiphy_write
                0xfff90778                mii_parse_88E1011_psr
 .text          0xfff914fc       0xc4 drivers/libdrivers.a(ns16550.o)
                0xfff91574                NS16550_putc
                0xfff914fc                NS16550_init
                0xfff915ac                NS16550_tstc
                0xfff91590                NS16550_getc
                0xfff91538                NS16550_reinit
 .text          0xfff915c0      0x9d0 common/libcommon.a(main.o)
                0xfff919e0                run_command
                0xfff91ee8                do_run
                0xfff917e8                readline
                0xfff915c4                main_loop
 .text          0xfff91f90      0x1e8 common/libcommon.a(cmd_autoscript.o)
                0xfff9210c                do_autoscript
                0xfff91f94                autoscript
 .text          0xfff92178      0x290 common/libcommon.a(cmd_bdinfo.o)
                0xfff9221c                do_bdinfo
 .text          0xfff92408       0xb4 common/libcommon.a(cmd_boot.o)
                0xfff9240c                do_go
 .text          0xfff924bc      0xf6c common/libcommon.a(cmd_bootm.o)
                0xfff92518                print_image_hdr
                0xfff924c0                do_bootd
                0xfff92ad4                gunzip
                0xfff92c4c                do_bootm
                0xfff929dc                do_iminfo
 .text          0xfff93428       0xf4 common/libcommon.a(cmd_console.o)
                0xfff9342c                do_coninfo
 .text          0xfff9351c      0xd18 common/libcommon.a(cmd_flash.o)
                0xfff93a4c                do_flinfo
                0xfff93b24                flash_sect_erase
                0xfff93f5c                do_protect
                0xfff93c30                do_flerase
                0xfff93e28                flash_sect_protect
 .text          0xfff94234      0x914 common/libcommon.a(cmd_i2c.o)
                0xfff94598                do_i2c_crc
                0xfff94920                do_i2c_nm
                0xfff9444c                do_i2c_mw
                0xfff94964                do_i2c_probe
                0xfff94940                do_i2c_mm
                0xfff94238                do_i2c_md
                0xfff94a14                do_i2c_loop
 .text          0xfff94b48      0x38c common/libcommon.a(cmd_itest.o)
                0xfff94c00                binary_test
                0xfff94e0c                do_itest
 .text          0xfff94ed4      0xef0 common/libcommon.a(cmd_load.o)
                0xfff95580                k_data_init
                0xfff95358                s1_sendpacket
                0xfff95754                handle_send_packet
                0xfff9564c                k_data_restore
                0xfff9542c                send_nack
                0xfff9596c                do_load_serial_bin
                0xfff956c4                k_data_char
                0xfff95324                chk1
                0xfff955d4                k_data_save
                0xfff952f4                ktrans
                0xfff9529c                send_pad
                0xfff953a0                send_ack
                0xfff94ed8                do_load_serial
 .text          0xfff95dc4      0xcc0 common/libcommon.a(cmd_mem.o)
                0xfff964a0                do_mem_base
                0xfff96068                do_mem_mw
                0xfff969a8                do_mem_crc
                0xfff96964                do_mem_nm
                0xfff96984                do_mem_mm
                0xfff9633c                do_mem_cp
                0xfff96658                do_mem_mtest
                0xfff96174                do_mem_cmp
                0xfff95dc4                cmd_get_data_size
                0xfff96510                do_mem_loop
                0xfff95e58                do_mem_md
 .text          0xfff96a84      0x7dc common/libcommon.a(cmd_mii.o)
                0xfff96a88                MII_dump_0_to_5
                0xfff96d94                do_mii
 .text          0xfff97260       0xb8 common/libcommon.a(cmd_misc.o)
                0xfff97264                do_sleep
 .text          0xfff97318      0x3b8 common/libcommon.a(cmd_net.o)
                0xfff975dc                do_rarpb
                0xfff9761c                do_ping
                0xfff975f0                do_tftpb
                0xfff97604                do_bootp
                0xfff975c8                do_nfs
 .text          0xfff976d0      0xa84 common/libcommon.a(cmd_nvedit.o)
                0xfff97f34                getenv
                0xfff97968                _do_setenv
                0xfff97fec                getenv_r
                0xfff9777c                do_printenv
                0xfff97e68                setenv
                0xfff980f8                do_saveenv
                0xfff97ec8                do_setenv
 .text          0xfff98154     0x125c common/libcommon.a(cmd_pci.o)
                0xfff9835c                pci_header_show
                0xfff98ca8                pciinfo
                0xfff98fbc                do_pci
                0xfff982c0                pci_header_show_brief
 .text          0xfff993b0      0x8b4 common/libcommon.a(command.o)
                0xfff993fc                do_echo
                0xfff99954                do_exit
                0xfff99994                find_cmd
                0xfff994a8                do_test
                0xfff99a68                do_help
                0xfff993b4                do_version
 .text          0xfff99c64      0x8f4 common/libcommon.a(console.o)
                0xfff9a394                console_init_r
                0xfff9a090                printf
                0xfff9a2ac                console_assign
                0xfff99fa8                getc
                0xfff9a054                puts
                0xfff9a29c                dbg
                0xfff99d40                serial_printf
                0xfff99e1c                ftstc
                0xfff99f2c                fprintf
                0xfff99fe0                tstc
                0xfff9a10c                vprintf
                0xfff9a150                ctrlc
                0xfff9a018                putc
                0xfff9a1d4                disable_ctrlc
                0xfff99dc0                fgetc
                0xfff9a21c                had_ctrlc
                0xfff99e78                fputc
                0xfff9a378                console_init_f
                0xfff9a25c                clear_ctrlc
                0xfff99ed4                fputs
 .text          0xfff9a558      0x190 common/libcommon.a(devices.o)
                0xfff9a55c                device_register
                0xfff9a6a4                devices_done
                0xfff9a5ac                devices_init
 .text          0xfff9a6e8      0x204 common/libcommon.a(env_common.o)
                0xfff9a7e8                env_get_addr
                0xfff9a840                env_relocate
                0xfff9a6ec                env_crc_update
                0xfff9a794                env_get_char_memory
 .text          0xfff9a8ec      0x1f8 common/libcommon.a(env_flash.o)
                0xfff9aa98                env_relocate_spec
                0xfff9a988                saveenv
                0xfff9a8ec                env_get_char_spec
                0xfff9a904                env_init
 .text          0xfff9aae4       0xf0 common/libcommon.a(exports.o)
                0xfff9ab04                jumptable_init
                0xfff9aaf0                get_version
 .text          0xfff9abd4      0x438 common/libcommon.a(flash.o)
                0xfff9ad60                flash_write
                0xfff9abd4                flash_protect
                0xfff9acd4                addr2info
                0xfff9af18                flash_perror
 .text          0xfff9b00c     0x223c common/libcommon.a(hush.o)
                0xfff9b954                new_pipe
                0xfff9be88                mapset
                0xfff9d160                parse_string_outer
                0xfff9bee0                update_ifs_map
                0xfff9d0f4                parse_file_outer
                0xfff9b1e4                simple_itoa
                0xfff9bb3c                reserved_word
                0xfff9bf70                u_boot_hush_start
 .text          0xfff9d248      0x53c common/libcommon.a(lists.o)
                0xfff9d2d4                DisposeHandle
                0xfff9d448                ListDispose
                0xfff9d468                ListInsertItems
                0xfff9d430                ListSetAllocationPolicy
                0xfff9d75c                ListGetItemSize
                0xfff9d748                ListGetDataPtr
                0xfff9d248                NewHandle
                0xfff9d320                SetHandleSize
                0xfff9d67c                ListInsertItem
                0xfff9d310                GetHandleSize
                0xfff9d770                ListNumItems
                0xfff9d704                ListGetPtrToItem
                0xfff9d3c8                ListCreate
                0xfff9d6a0                ListGetItems
 .text          0xfff9d784      0x7d8 common/libcommon.a(miiphyutil.o)
                0xfff9dde0                miiphy_speed
                0xfff9dc50                miiphy_info
                0xfff9dd04                miiphy_reset
                0xfff9d8f4                miiphy_set_current_dev
                0xfff9dbbc                miiphy_listdev
                0xfff9d9d4                miiphy_read
                0xfff9d984                miiphy_get_current_dev
                0xfff9dea0                miiphy_duplex
                0xfff9dac8                miiphy_write
                0xfff9d7d8                miiphy_register
                0xfff9d788                miiphy_init
 .text          0xfff9df5c      0x354 common/libcommon.a(s_record.o)
                0xfff9e00c                srec_decode
 .text          0xfff9e2b0      0x108 lib_generic/libgeneric.a(display_options.o)
                0xfff9e2b4                display_options
                0xfff9e300                print_size
 .text          0xfff9e3b8      0x6f0 cpu/mpc85xx/libmpc85xx.a(i2c.o)
                0xfff9e784                i2c_write
                0xfff9ea00                i2c_probe
                0xfff9ea48                i2c_reg_read
                0xfff9e42c                i2c_read
                0xfff9ea78                i2c_reg_write
                0xfff9e3b8                i2c_init
 .text          0xfff9eaa8       0x6c lib_ppc/libppc.a(cache.o)
                0xfff9eaa8                flush_cache
 *(.fixup)
 *(.got1)
                0xfff9eb14                _etext = .
                0xfff9eb14                PROVIDE (etext, .)

.rodata         0xfff9eb14     0x65a5
 *(.rodata)
 .rodata        0xfff9eb14      0x400 lib_generic/crc32.o
 .rodata        0xfff9ef14       0x74 lib_generic/zlib.o
 .rodata        0xfff9ef88       0x20 board/mpc8548pc/libmpc8548pc.a(mpc8548pc.o)
 .rodata        0xfff9efa8       0x28 net/libnet.a(net.o)
 .rodata        0xfff9efd0       0x14 net/libnet.a(tftp.o)
 .rodata        0xfff9efe4        0x8 net/libnet.a(eth.o)
 .rodata        0xfff9efec       0x38 net/libnet.a(nfs.o)
 .rodata        0xfff9f024       0xa8 common/libcommon.a(cmd_bootm.o)
 .rodata        0xfff9f0cc       0x30 common/libcommon.a(cmd_itest.o)
 .rodata        0xfff9f0fc       0x24 common/libcommon.a(cmd_nvedit.o)
 .rodata        0xfff9f120       0x28 common/libcommon.a(s_record.o)
 *(.rodata1)
 *(.rodata.str1.4)
 .rodata.str1.4
                0xfff9f148      0x2a8 cpu/mpc85xx/traps.o
                                0x2ac (size before relaxing)
 .rodata.str1.4
                0xfff9f3f0       0x4a cpu/mpc85xx/cpu_init.o
                                 0x4c (size before relaxing)
 *fill*         0xfff9f43a        0x2 00
 .rodata.str1.4
                0xfff9f43c      0x164 cpu/mpc85xx/cpu.o
 .rodata.str1.4
                0xfff9f5a0       0x24 lib_ppc/extable.o
 .rodata.str1.4
                0xfff9f5c4      0x20d lib_generic/zlib.o
                                0x214 (size before relaxing)
 *fill*         0xfff9f7d1        0x3 00
 .rodata.str1.4
                0xfff9f7d4       0x57 lib_generic/libgeneric.a(vsprintf.o)
                                 0x58 (size before relaxing)
 *fill*         0xfff9f82b        0x1 00
 .rodata.str1.4
                0xfff9f82c      0x35c board/mpc8548pc/libmpc8548pc.a(mpc8548pc.o)
                                0x368 (size before relaxing)
 .rodata.str1.4
                0xfff9fb88       0xc8 lib_ppc/libppc.a(board.o)
                                 0xd0 (size before relaxing)
 .rodata.str1.4
                0xfff9fc50      0x241 net/libnet.a(net.o)
                                0x244 (size before relaxing)
 *fill*         0xfff9fe91        0x3 00
 .rodata.str1.4
                0xfff9fe94      0x1cb net/libnet.a(tftp.o)
                                0x1e8 (size before relaxing)
 *fill*         0xfffa005f        0x1 00
 .rodata.str1.4
                0xfffa0060       0x84 net/libnet.a(bootp.o)
                                 0xb8 (size before relaxing)
 .rodata.str1.4
                0xfffa00e4       0x13 net/libnet.a(rarp.o)
                                 0x4c (size before relaxing)
 *fill*         0xfffa00f7        0x1 00
 .rodata.str1.4
                0xfffa00f8       0xf0 net/libnet.a(eth.o)
                                0x11c (size before relaxing)
 .rodata.str1.4
                0xfffa01e8      0x101 net/libnet.a(nfs.o)
                                0x1a0 (size before relaxing)
 *fill*         0xfffa02e9        0x3 00
 .rodata.str1.4
                0xfffa02ec      0x28a drivers/libdrivers.a(cfi_flash.o)
                                0x298 (size before relaxing)
 *fill*         0xfffa0576        0x2 00
 .rodata.str1.4
                0xfffa0578       0x7e drivers/libdrivers.a(pci.o)
                                 0x80 (size before relaxing)
 *fill*         0xfffa05f6        0x2 00
 .rodata.str1.4
                0xfffa05f8      0x13b drivers/libdrivers.a(tsec.o)
                                0x150 (size before relaxing)
 *fill*         0xfffa0733        0x1 00
 .rodata.str1.4
                0xfffa0734       0xe4 common/libcommon.a(main.o)
 .rodata.str1.4
                0xfffa0818       0xf6 common/libcommon.a(cmd_autoscript.o)
                                 0xf8 (size before relaxing)
 *fill*         0xfffa090e        0x2 00
 .rodata.str1.4
                0xfffa0910      0x139 common/libcommon.a(cmd_bdinfo.o)
                                0x13c (size before relaxing)
 *fill*         0xfffa0a49        0x3 00
 .rodata.str1.4
                0xfffa0a4c      0x10b common/libcommon.a(cmd_boot.o)
                                0x118 (size before relaxing)
 *fill*         0xfffa0b57        0x1 00
 .rodata.str1.4
                0xfffa0b58      0x8fd common/libcommon.a(cmd_bootm.o)
                                0x934 (size before relaxing)
 *fill*         0xfffa1455        0x3 00
 .rodata.str1.4
                0xfffa1458       0x70 common/libcommon.a(cmd_console.o)
                                 0x74 (size before relaxing)
 .rodata.str1.4
                0xfffa14c8      0x744 common/libcommon.a(cmd_flash.o)
                                0x780 (size before relaxing)
 .rodata.str1.4
                0xfffa1c0c      0x42d common/libcommon.a(cmd_i2c.o)
                                0x444 (size before relaxing)
 *fill*         0xfffa2039        0x3 00
 .rodata.str1.4
                0xfffa203c       0xce common/libcommon.a(cmd_itest.o)
                                 0xdc (size before relaxing)
 *fill*         0xfffa210a        0x2 00
 .rodata.str1.4
                0xfffa210c      0x30d common/libcommon.a(cmd_load.o)
                                0x32c (size before relaxing)
 *fill*         0xfffa2419        0x3 00
 .rodata.str1.4
                0xfffa241c      0x609 common/libcommon.a(cmd_mem.o)
                                0x648 (size before relaxing)
 *fill*         0xfffa2a25        0x3 00
 .rodata.str1.4
                0xfffa2a28      0x7e3 common/libcommon.a(cmd_mii.o)
                                0x80c (size before relaxing)
 *fill*         0xfffa320b        0x1 00
 .rodata.str1.4
                0xfffa320c       0x70 common/libcommon.a(cmd_misc.o)
                                 0x7c (size before relaxing)
 .rodata.str1.4
                0xfffa327c      0x22e common/libcommon.a(cmd_net.o)
                                0x27c (size before relaxing)
 *fill*         0xfffa34aa        0x2 00
 .rodata.str1.4
                0xfffa34ac      0x2e9 common/libcommon.a(cmd_nvedit.o)
                                0x384 (size before relaxing)
 *fill*         0xfffa3795        0x3 00
 .rodata.str1.4
                0xfffa3798      0xddf common/libcommon.a(cmd_pci.o)
                                0xe18 (size before relaxing)
 *fill*         0xfffa4577        0x1 00
 .rodata.str1.4
                0xfffa4578      0x322 common/libcommon.a(command.o)
                                0x34c (size before relaxing)
 *fill*         0xfffa489a        0x2 00
 .rodata.str1.4
                0xfffa489c       0x75 common/libcommon.a(console.o)
                                 0x7c (size before relaxing)
 *fill*         0xfffa4911        0x3 00
 .rodata.str1.4
                0xfffa4914       0x2f common/libcommon.a(devices.o)
                                 0x48 (size before relaxing)
 *fill*         0xfffa4943        0x1 00
 .rodata.str1.4
                0xfffa4944       0x33 common/libcommon.a(env_common.o)
                                 0x34 (size before relaxing)
 *fill*         0xfffa4977        0x1 00
 .rodata.str1.4
                0xfffa4978       0x31 common/libcommon.a(env_flash.o)
                                 0x3c (size before relaxing)
 *fill*         0xfffa49a9        0x3 00
 .rodata.str1.4
                0xfffa49ac      0x120 common/libcommon.a(flash.o)
 .rodata.str1.4
                0xfffa4acc      0x441 common/libcommon.a(hush.o)
                                0x4a4 (size before relaxing)
 *fill*         0xfffa4f0d        0x3 00
 .rodata.str1.4
                0xfffa4f10      0x189 common/libcommon.a(miiphyutil.o)
                                0x190 (size before relaxing)
 *fill*         0xfffa5099        0x3 00
 .rodata.str1.4
                0xfffa509c       0x1d lib_generic/libgeneric.a(display_options.o)
                                 0x20 (size before relaxing)
 *(.eh_frame)

.fini
 *(.fini)

.ctors
 *(.ctors)

.dtors
 *(.dtors)
                0xfffa5100                . = ((. + 0xff) & 0xffffff00)
                0xfffa5100                _erotext = .
                0xfffa5100                PROVIDE (erotext, .)

.reloc          0xfffa5100     0x1120
 *(.got)
                0xfffa5100                _GOT2_TABLE_ = .
 *(.got2)
 .got2          0xfffa5100       0x24 cpu/mpc85xx/start.o
 .got2          0xfffa5124       0x60 cpu/mpc85xx/traps.o
 .got2          0xfffa5184        0x8 cpu/mpc85xx/interrupts.o
 .got2          0xfffa518c       0x10 cpu/mpc85xx/cpu_init.o
 .got2          0xfffa519c       0x64 cpu/mpc85xx/cpu.o
 .got2          0xfffa5200       0x2c common/dlmalloc.o
 .got2          0xfffa522c        0x4 lib_generic/crc32.o
 .got2          0xfffa5230       0x10 lib_ppc/extable.o
 .got2          0xfffa5240       0x8c lib_generic/zlib.o
 .got2          0xfffa52cc       0x10 lib_generic/libgeneric.a(vsprintf.o)
 .got2          0xfffa52dc        0x8 lib_generic/libgeneric.a(string.o)
 .got2          0xfffa52e4       0xb8 board/mpc8548pc/libmpc8548pc.a(mpc8548pc.o)
 .got2          0xfffa539c       0x7c lib_ppc/libppc.a(board.o)
 .got2          0xfffa5418      0x130 net/libnet.a(net.o)
 .got2          0xfffa5548       0xc0 net/libnet.a(tftp.o)
 .got2          0xfffa5608       0x74 net/libnet.a(bootp.o)
 .got2          0xfffa567c       0x30 net/libnet.a(rarp.o)
 .got2          0xfffa56ac       0x54 net/libnet.a(eth.o)
 .got2          0xfffa5700       0xc8 net/libnet.a(nfs.o)
 .got2          0xfffa57c8       0x74 drivers/libdrivers.a(cfi_flash.o)
 .got2          0xfffa583c       0x1c drivers/libdrivers.a(pci.o)
 .got2          0xfffa5858       0x18 drivers/libdrivers.a(pci_indirect.o)
 .got2          0xfffa5870        0x4 drivers/libdrivers.a(serial.o)
 .got2          0xfffa5874       0x60 drivers/libdrivers.a(tsec.o)
 .got2          0xfffa58d4       0x3c common/libcommon.a(main.o)
 .got2          0xfffa5910       0x20 common/libcommon.a(cmd_autoscript.o)
 .got2          0xfffa5930       0x50 common/libcommon.a(cmd_bdinfo.o)
 .got2          0xfffa5980        0xc common/libcommon.a(cmd_boot.o)
 .got2          0xfffa598c      0x16c common/libcommon.a(cmd_bootm.o)
 .got2          0xfffa5af8       0x18 common/libcommon.a(cmd_console.o)
 .got2          0xfffa5b10       0x64 common/libcommon.a(cmd_flash.o)
 .got2          0xfffa5b74       0x74 common/libcommon.a(cmd_i2c.o)
 .got2          0xfffa5be8       0x18 common/libcommon.a(cmd_itest.o)
 .got2          0xfffa5c00       0x9c common/libcommon.a(cmd_load.o)
 .got2          0xfffa5c9c       0x80 common/libcommon.a(cmd_mem.o)
 .got2          0xfffa5d1c       0x98 common/libcommon.a(cmd_mii.o)
 .got2          0xfffa5db4        0x4 common/libcommon.a(cmd_misc.o)
 .got2          0xfffa5db8       0x68 common/libcommon.a(cmd_net.o)
 .got2          0xfffa5e20       0x64 common/libcommon.a(cmd_nvedit.o)
 .got2          0xfffa5e84      0x178 common/libcommon.a(cmd_pci.o)
 .got2          0xfffa5ffc       0x54 common/libcommon.a(command.o)
 .got2          0xfffa6050       0x34 common/libcommon.a(console.o)
 .got2          0xfffa6084       0x20 common/libcommon.a(devices.o)
 .got2          0xfffa60a4       0x14 common/libcommon.a(env_common.o)
 .got2          0xfffa60b8       0x18 common/libcommon.a(env_flash.o)
 .got2          0xfffa60d0       0x28 common/libcommon.a(exports.o)
 .got2          0xfffa60f8       0x2c common/libcommon.a(flash.o)
 .got2          0xfffa6124       0xa8 common/libcommon.a(hush.o)
 .got2          0xfffa61cc       0x3c common/libcommon.a(miiphyutil.o)
 .got2          0xfffa6208        0x4 common/libcommon.a(s_record.o)
 .got2          0xfffa620c       0x14 lib_generic/libgeneric.a(display_options.o)
                0xfffa6220                _FIXUP_TABLE_ = .
 *(.fixup)
                0x00000448                __got2_entries = ((_FIXUP_TABLE_ - _GOT2_TABLE_) >> 0x2)
                0x00000000                __fixup_entries = ((. - _FIXUP_TABLE_) >> 0x2)

.data           0xfffa6220      0xc18
 *(.data)
 .data          0xfffa6220        0xc common/dlmalloc.o
 .data          0xfffa622c      0x27c lib_generic/zlib.o
 .data          0xfffa64a8      0x100 lib_generic/libgeneric.a(ctype.o)
                0xfffa64a8                _ctype
 .data          0xfffa65a8        0x4 net/libnet.a(nfs.o)
 .data          0xfffa65ac        0x8 drivers/libdrivers.a(cfi_flash.o)
 .data          0xfffa65b4       0x10 drivers/libdrivers.a(serial.o)
 .data          0xfffa65c4      0x168 drivers/libdrivers.a(tsec.o)
 .data          0xfffa672c       0x10 common/libcommon.a(main.o)
 .data          0xfffa673c        0x8 common/libcommon.a(cmd_i2c.o)
 .data          0xfffa6744        0x4 common/libcommon.a(cmd_load.o)
 .data          0xfffa6748      0x698 common/libcommon.a(env_common.o)
                0xfffa6748                default_environment
 .data          0xfffa6de0        0x4 common/libcommon.a(env_flash.o)
 .data          0xfffa6de4       0x28 common/libcommon.a(hush.o)
 *(.data1)
 *(.sdata)
 .sdata         0xfffa6e0c        0x4 lib_ppc/extable.o
                0xfffa6e0c                ex_tab_message
 .sdata         0xfffa6e10        0x4 lib_generic/zlib.o
                0xfffa6e10                zlib_version
 .sdata         0xfffa6e14        0xc net/libnet.a(net.o)
                0xfffa6e18                NetBcastAddr
                0xfffa6e14                NetOurNativeVLAN
                0xfffa6e16                NetOurVLAN
 .sdata         0xfffa6e20        0x4 common/libcommon.a(cmd_bootm.o)
                0xfffa6e20                load_addr
 .sdata         0xfffa6e24        0x4 common/libcommon.a(cmd_mem.o)
                0xfffa6e24                dp_last_length
 .sdata         0xfffa6e28        0x1 common/libcommon.a(cmd_pci.o)
                0xfffa6e28                ShortPCIListing
 *fill*         0xfffa6e29        0x3 00
 .sdata         0xfffa6e2c        0x4 common/libcommon.a(env_common.o)
                0xfffa6e2c                env_get_char
 .sdata         0xfffa6e30        0x8 common/libcommon.a(env_flash.o)
                0xfffa6e34                env_name_spec
                0xfffa6e30                env_ptr
 *(.sdata2)
 *(.dynamic)

.data.rel.local
                0xfffa6e38      0x89c
 .data.rel.local
                0xfffa6e38      0x408 common/dlmalloc.o
 .data.rel.local
                0xfffa7240       0x20 lib_generic/zlib.o
                0xfffa7240                z_errmsg
 .data.rel.local
                0xfffa7260        0x4 lib_ppc/libppc.a(board.o)
 .data.rel.local
                0xfffa7264       0xc0 drivers/libdrivers.a(tsec.o)
                0xfffa72f4                phy_info_M88E1111S
                0xfffa730c                phy_info_M88E1011S
                0xfffa72ac                phy_info_rtl821x
                0xfffa727c                phy_info_dm9161
                0xfffa72c4                phy_info_cis8201
                0xfffa7294                phy_info_rtl8201cp
                0xfffa72dc                phy_info_cis8204
 .data.rel.local
                0xfffa7324       0x68 common/libcommon.a(cmd_itest.o)
                0xfffa7324                op_table
 .data.rel.local
                0xfffa738c      0x2b8 common/libcommon.a(cmd_mii.o)
                0xfffa74ac                reg_3_desc_tbl
                0xfffa759c                reg_0_desc_tbl
                0xfffa741c                reg_4_desc_tbl
                0xfffa7614                reg_0_5_desc_tbl
                0xfffa738c                reg_5_desc_tbl
                0xfffa74dc                reg_1_desc_tbl
                0xfffa74d0                reg_2_desc_tbl
 .data.rel.local
                0xfffa7644        0xc common/libcommon.a(devices.o)
                0xfffa7644                stdio_names
 .data.rel.local
                0xfffa7650       0x84 common/libcommon.a(hush.o)

.data.rel       0xfffa76d4      0x354
 .data.rel      0xfffa76d4       0x34 lib_ppc/libppc.a(board.o)
                0xfffa76d4                init_sequence
 .data.rel      0xfffa7708      0x2f0 drivers/libdrivers.a(tsec.o)
                0xfffa7708                phy_info
 .data.rel      0xfffa79f8       0x30 common/libcommon.a(cmd_mii.o)
                0xfffa79f8                desc_and_len_tbl
                0xfffa7a28                _edata = .
                0xfffa7a28                PROVIDE (edata, .)
                0xfffa7a28                . = .
                0xfffa7a28                __u_boot_cmd_start = .

.u_boot_cmd     0xfffa7a28      0x4c8
 *(.u_boot_cmd)
 .u_boot_cmd    0xfffa7a28       0x18 common/libcommon.a(cmd_autoscript.o)
                0xfffa7a28                __u_boot_cmd_autoscr
 .u_boot_cmd    0xfffa7a40       0x18 common/libcommon.a(cmd_bdinfo.o)
                0xfffa7a40                __u_boot_cmd_bdinfo
 .u_boot_cmd    0xfffa7a58       0x30 common/libcommon.a(cmd_boot.o)
                0xfffa7a58                __u_boot_cmd_reset
                0xfffa7a70                __u_boot_cmd_go
 .u_boot_cmd    0xfffa7a88       0x78 common/libcommon.a(cmd_bootm.o)
                0xfffa7ae8                __u_boot_cmd_bootm
                0xfffa7aa0                __u_boot_cmd_iminfo
                0xfffa7ab8                __u_boot_cmd_bootd
                0xfffa7ad0                __u_boot_cmd_boot
                0xfffa7a88                __u_boot_cmd_imls
 .u_boot_cmd    0xfffa7b00       0x18 common/libcommon.a(cmd_console.o)
                0xfffa7b00                __u_boot_cmd_coninfo
 .u_boot_cmd    0xfffa7b18       0x48 common/libcommon.a(cmd_flash.o)
                0xfffa7b48                __u_boot_cmd_flinfo
                0xfffa7b30                __u_boot_cmd_erase
                0xfffa7b18                __u_boot_cmd_protect
 .u_boot_cmd    0xfffa7b60       0xa8 common/libcommon.a(cmd_i2c.o)
                0xfffa7b90                __u_boot_cmd_icrc32
                0xfffa7ba8                __u_boot_cmd_imw
                0xfffa7bd8                __u_boot_cmd_imm
                0xfffa7bf0                __u_boot_cmd_imd
                0xfffa7b60                __u_boot_cmd_iloop
                0xfffa7b78                __u_boot_cmd_iprobe
                0xfffa7bc0                __u_boot_cmd_inm
 .u_boot_cmd    0xfffa7c08       0x18 common/libcommon.a(cmd_itest.o)
                0xfffa7c08                __u_boot_cmd_itest
 .u_boot_cmd    0xfffa7c20       0x30 common/libcommon.a(cmd_load.o)
                0xfffa7c20                __u_boot_cmd_loadb
                0xfffa7c38                __u_boot_cmd_loads
 .u_boot_cmd    0xfffa7c50       0xf0 common/libcommon.a(cmd_mem.o)
                0xfffa7d28                __u_boot_cmd_md
                0xfffa7cb0                __u_boot_cmd_cmp
                0xfffa7ce0                __u_boot_cmd_mw
                0xfffa7c68                __u_boot_cmd_loop
                0xfffa7c80                __u_boot_cmd_base
                0xfffa7d10                __u_boot_cmd_mm
                0xfffa7c98                __u_boot_cmd_crc32
                0xfffa7cf8                __u_boot_cmd_nm
                0xfffa7c50                __u_boot_cmd_mtest
                0xfffa7cc8                __u_boot_cmd_cp
 .u_boot_cmd    0xfffa7d40       0x18 common/libcommon.a(cmd_mii.o)
                0xfffa7d40                __u_boot_cmd_mii
 .u_boot_cmd    0xfffa7d58       0x18 common/libcommon.a(cmd_misc.o)
                0xfffa7d58                __u_boot_cmd_sleep
 .u_boot_cmd    0xfffa7d70       0x78 common/libcommon.a(cmd_net.o)
                0xfffa7d88                __u_boot_cmd_nfs
                0xfffa7d70                __u_boot_cmd_ping
                0xfffa7da0                __u_boot_cmd_rarpboot
                0xfffa7db8                __u_boot_cmd_tftpboot
                0xfffa7dd0                __u_boot_cmd_bootp
 .u_boot_cmd    0xfffa7de8       0x60 common/libcommon.a(cmd_nvedit.o)
                0xfffa7de8                __u_boot_cmd_run
                0xfffa7e00                __u_boot_cmd_saveenv
                0xfffa7e30                __u_boot_cmd_printenv
                0xfffa7e18                __u_boot_cmd_setenv
 .u_boot_cmd    0xfffa7e48       0x18 common/libcommon.a(cmd_pci.o)
                0xfffa7e48                __u_boot_cmd_pci
 .u_boot_cmd    0xfffa7e60       0x90 common/libcommon.a(command.o)
                0xfffa7e90                __u_boot_cmd_exit
                0xfffa7ec0                __u_boot_cmd_echo
                0xfffa7e60                __u_boot_cmd_question_mark
                0xfffa7ed8                __u_boot_cmd_version
                0xfffa7e78                __u_boot_cmd_help
                0xfffa7ea8                __u_boot_cmd_test
                0xfffa7ef0                __u_boot_cmd_end = .
                0xfffa7ef0                . = .
                0xfffa7ef0                __start___ex_table = .

__ex_table
 *(__ex_table)
                0xfffa7ef0                __stop___ex_table = .
                0xfffa7f00                . = ALIGN (0x100)
                0xfffa7f00                __init_begin = .

.text.init
 *(.text.init)

.data.init
 *(.data.init)
                0xfffa7f00                . = ALIGN (0x100)
                0xfffa7f00                __init_end = .
                0xfffa7f00                __bss_start = .

.bss            0xfffa7f00     0x4b28
 *(.sbss)
 .sbss          0xfffa7f00        0x4 cpu/mpc85xx/interrupts.o
                0xfffa7f00                timestamp
 .sbss          0xfffa7f04        0x4 cpu/mpc85xx/interrupts.o
                                  0x0 (size before relaxing)
                0xfffa7f04                decrementer_count
 .sbss          0xfffa7f08       0x14 common/dlmalloc.o
 .sbss          0xfffa7f1c       0x18 lib_generic/zlib.o
 .sbss          0xfffa7f34        0x4 lib_generic/libgeneric.a(string.o)
                                  0x0 (size before relaxing)
                0xfffa7f34                ___strtok
 .sbss          0xfffa7f38       0x10 lib_ppc/libppc.a(board.o)
                                  0xc (size before relaxing)
                0xfffa7f44                monitor_flash_len
 .sbss          0xfffa7f48       0x8c net/libnet.a(net.o)
                                 0x48 (size before relaxing)
                0xfffa7f90                NetArpWaitTry
                0xfffa7f94                NetArpWaitPacketMAC
                0xfffa7f98                NetOurEther
                0xfffa7fa0                NetOurIP
                0xfffa7fa4                NetPingIP
                0xfffa7fa8                NetServerIP
                0xfffa7fac                NetArpWaitTxPacketSize
                0xfffa7fb0                NetArpWaitReplyIP
                0xfffa7fb4                NetArpWaitTxPacket
                0xfffa7fb8                NetArpWaitPacketIP
                0xfffa7fbc                NetState
                0xfffa7f58                NetServerEther
                0xfffa7f68                NetOurSubnetMask
                0xfffa7f5e                NetBootFileSize
                0xfffa7fc0                NetIPID
                0xfffa7fc4                NetRxPkt
                0xfffa7f64                NetOurGatewayIP
                0xfffa7f50                NetEtherNullAddr
                0xfffa7f4c                NetRestartWrap
                0xfffa7fc8                NetRxPktLen
                0xfffa7f48                NetTxPacket
                0xfffa7fcc                NetBootFileXferSize
                0xfffa7f60                NetOurDNSIP
                0xfffa7fd0                NetArpWaitTimerStart
 .sbss          0xfffa7fd4       0x24 net/libnet.a(tftp.o)
 .sbss          0xfffa7ff8        0x8 net/libnet.a(bootp.o)
                                  0x0 (size before relaxing)
                0xfffa7ff8                BootpTry
                0xfffa7ffc                BootpID
 .sbss          0xfffa8000        0x4 net/libnet.a(rarp.o)
                                  0x0 (size before relaxing)
                0xfffa8000                RarpTry
 .sbss          0xfffa8004        0xc net/libnet.a(eth.o)
 .sbss          0xfffa8010       0x30 net/libnet.a(nfs.o)
 .sbss          0xfffa8040        0x4 drivers/libdrivers.a(pci.o)
 .sbss          0xfffa8044        0xc drivers/libdrivers.a(tsec.o)
 .sbss          0xfffa8050       0x18 common/libcommon.a(cmd_i2c.o)
 .sbss          0xfffa8068       0x3c common/libcommon.a(cmd_load.o)
                                 0x20 (size before relaxing)
                0xfffa8088                his_pad_char
                0xfffa808c                os_data_count
                0xfffa8090                os_data_init
                0xfffa8094                send_ptr
                0xfffa8098                os_data_char
                0xfffa809c                his_eol
                0xfffa809d                his_quote
                0xfffa80a0                his_pad_count
 .sbss          0xfffa80a4       0x14 common/libcommon.a(cmd_mem.o)
                                  0x4 (size before relaxing)
                0xfffa80a8                dp_last_size
                0xfffa80ac                dp_last_addr
                0xfffa80b0                mm_last_size
                0xfffa80b4                mm_last_addr
 .sbss          0xfffa80b8       0x18 common/libcommon.a(cmd_mii.o)
                                  0x0 (size before relaxing)
                0xfffa80b8                last_reg_hi
                0xfffa80bc                last_data
                0xfffa80c0                last_addr_hi
                0xfffa80c4                last_reg_lo
                0xfffa80c8                last_op
                0xfffa80cc                last_addr_lo
 .sbss          0xfffa80d0        0x8 common/libcommon.a(console.o)
 .sbss          0xfffa80d8        0x4 common/libcommon.a(devices.o)
                0xfffa80d8                devlist
 .sbss          0xfffa80dc       0x18 common/libcommon.a(hush.o)
                                 0x10 (size before relaxing)
                0xfffa80ec                nesting_level
                0xfffa80f0                last_return_code
 .sbss          0xfffa80f4        0xc common/libcommon.a(miiphyutil.o)
 *(.scommon)
 *(.dynbss)
 *(.bss)
 .bss           0xfffa8100       0x28 common/dlmalloc.o
 .bss           0xfffa8128     0x1090 lib_generic/zlib.o
 .bss           0xfffa91b8       0xd4 board/mpc8548pc/libmpc8548pc.a(mpc8548pc.o)
 .bss           0xfffa928c       0x80 net/libnet.a(net.o)
                0xfffa92ec                NetOurNISDomain
                0xfffa92cc                NetOurHostName
                0xfffa928c                NetOurRootPath
 .bss           0xfffa930c       0x10 net/libnet.a(tftp.o)
 .bss           0xfffa931c      0x880 net/libnet.a(nfs.o)
 .bss           0xfffa9b9c       0x10 drivers/libdrivers.a(pci.o)
 *fill*         0xfffa9bac        0x4 00
 .bss           0xfffa9bb0       0x40 drivers/libdrivers.a(tsec.o)
 .bss           0xfffa9bf0       0x18 common/libcommon.a(cmd_load.o)
 .bss           0xfffa9c08        0xc common/libcommon.a(devices.o)
                0xfffa9c08                stdio_devices
 .bss           0xfffa9c14      0x240 common/libcommon.a(hush.o)
 *(COMMON)
 COMMON         0xfffa9e54     0x24d0 net/libnet.a(net.o)
                                  0x0 (size before relaxing)
                0xfffa9e54                NetRxPackets
                0xfffa9e64                BootFile
                0xfffa9ee4                NetArpWaitPacketBuf
                0xfffaa504                PktBuf
 COMMON         0xfffac324      0x590 drivers/libdrivers.a(cfi_flash.o)
                                  0x0 (size before relaxing)
                0xfffac324                flash_info
 COMMON         0xfffac8b4      0x100 common/libcommon.a(main.o)
                                  0x0 (size before relaxing)
                0xfffac8b4                console_buffer
 COMMON         0xfffac9b4       0x40 common/libcommon.a(cmd_bootm.o)
                                  0x0 (size before relaxing)
                0xfffac9b4                header
 COMMON         0xfffac9f4       0x34 common/libcommon.a(cmd_load.o)
                                  0x0 (size before relaxing)
                0xfffac9f4                os_data_header
                0xfffaca14                send_parms
                0xfffaca28                _end = .
                0xfffaca28                PROVIDE (end, .)
Address of section .text set to 0xfff80000
LOAD cpu/mpc85xx/start.o
LOAD cpu/mpc85xx/resetvec.o
START GROUP
LOAD lib_generic/libgeneric.a
LOAD board/mpc8548pc/libmpc8548pc.a
LOAD cpu/mpc85xx/libmpc85xx.a
LOAD lib_ppc/libppc.a
LOAD fs/cramfs/libcramfs.a
LOAD fs/fat/libfat.a
LOAD fs/fdos/libfdos.a
LOAD fs/jffs2/libjffs2.a
LOAD fs/reiserfs/libreiserfs.a
LOAD fs/ext2/libext2fs.a
LOAD net/libnet.a
LOAD disk/libdisk.a
LOAD rtc/librtc.a
LOAD dtt/libdtt.a
LOAD drivers/libdrivers.a
LOAD drivers/sk98lin/libsk98lin.a
LOAD post/libpost.a
LOAD post/cpu/libcpu.a
LOAD common/libcommon.a
END GROUP
LOAD /opt/mtwk/usr/local/gcc-3_4-e500-glibc-2.3.4-dp/powerpc-linux-gnuspe/lib/gcc/powerpc-linux-gnuspe/3.4.3/nof/libgcc.a
OUTPUT(u-boot elf32-powerpc)

.stab           0x00000000     0x2538
 .stab          0x00000000     0x1bfc cpu/mpc85xx/start.o
 .stab          0x00001bfc       0x48 board/mpc8548pc/init.o
                                 0x54 (size before relaxing)
 .stab          0x00001c44       0x24 cpu/mpc85xx/resetvec.o
                                 0x30 (size before relaxing)
 .stab          0x00001c68      0x7ec lib_ppc/libppc.a(ppcstring.o)
                                0x7f8 (size before relaxing)
 .stab          0x00002454       0xe4 lib_ppc/libppc.a(ticks.o)
                                 0xf0 (size before relaxing)

.PPC.EMB.apuinfo
                0x00000000       0x1c
 .PPC.EMB.apuinfo
                0x00000000       0x18 cpu/mpc85xx/start.o
 .PPC.EMB.apuinfo
                0x00000018       0x18 common/dlmalloc.o
 .PPC.EMB.apuinfo
                0x00000030       0x18 lib_generic/zlib.o
 .PPC.EMB.apuinfo
                0x00000048       0x18 lib_generic/libgeneric.a(vsprintf.o)
 .PPC.EMB.apuinfo
                0x00000060       0x18 net/libnet.a(net.o)
 .PPC.EMB.apuinfo
                0x00000078       0x18 net/libnet.a(eth.o)
 .PPC.EMB.apuinfo
                0x00000090       0x18 drivers/libdrivers.a(cfi_flash.o)
 .PPC.EMB.apuinfo
                0x000000a8       0x18 drivers/libdrivers.a(pci.o)
 .PPC.EMB.apuinfo
                0x000000c0       0x18 drivers/libdrivers.a(pci_auto.o)
 .PPC.EMB.apuinfo
                0x000000d8       0x18 drivers/libdrivers.a(tsec.o)
 .PPC.EMB.apuinfo
                0x000000f0       0x18 common/libcommon.a(main.o)
 .PPC.EMB.apuinfo
                0x00000108       0x18 common/libcommon.a(cmd_bdinfo.o)
 .PPC.EMB.apuinfo
                0x00000120       0x18 common/libcommon.a(cmd_boot.o)
 .PPC.EMB.apuinfo
                0x00000138       0x18 common/libcommon.a(cmd_bootm.o)
 .PPC.EMB.apuinfo
                0x00000150       0x18 common/libcommon.a(cmd_console.o)
 .PPC.EMB.apuinfo
                0x00000168       0x18 common/libcommon.a(cmd_i2c.o)
 .PPC.EMB.apuinfo
                0x00000180       0x18 common/libcommon.a(cmd_itest.o)
 .PPC.EMB.apuinfo
                0x00000198       0x18 common/libcommon.a(cmd_load.o)
 .PPC.EMB.apuinfo
                0x000001b0       0x18 common/libcommon.a(cmd_mem.o)
 .PPC.EMB.apuinfo
                0x000001c8       0x18 common/libcommon.a(cmd_pci.o)
 .PPC.EMB.apuinfo
                0x000001e0       0x18 common/libcommon.a(command.o)
 .PPC.EMB.apuinfo
                0x000001f8       0x18 common/libcommon.a(console.o)
 .PPC.EMB.apuinfo
                0x00000210       0x18 common/libcommon.a(flash.o)
 .PPC.EMB.apuinfo
                0x00000228       0x18 common/libcommon.a(hush.o)
 .PPC.EMB.apuinfo
                0x00000240       0x18 common/libcommon.a(lists.o)
 .PPC.EMB.apuinfo
                0x00000258       0x18 common/libcommon.a(miiphyutil.o)
 .PPC.EMB.apuinfo
                0x00000270       0x18 common/libcommon.a(s_record.o)
 .PPC.EMB.apuinfo
                0x00000288       0x18 cpu/mpc85xx/libmpc85xx.a(i2c.o)

.stabstr        0x00000000      0x122
 .stabstr       0x00000000      0x122 cpu/mpc85xx/start.o
                                  0x0 (size before relaxing)

.debug_abbrev   0x00000000     0x6034
 .debug_abbrev  0x00000000      0x190 cpu/mpc85xx/traps.o
 .debug_abbrev  0x00000190      0x208 cpu/mpc85xx/interrupts.o
 .debug_abbrev  0x00000398      0x170 cpu/mpc85xx/cpu_init.o
 .debug_abbrev  0x00000508      0x1e9 cpu/mpc85xx/cpu.o
 .debug_abbrev  0x000006f1      0x192 cpu/mpc85xx/speed.o
 .debug_abbrev  0x00000883      0x1ad cpu/mpc85xx/pci.o
 .debug_abbrev  0x00000a30      0x1c0 common/dlmalloc.o
 .debug_abbrev  0x00000bf0       0x90 lib_generic/crc32.o
 .debug_abbrev  0x00000c80      0x121 lib_ppc/extable.o
 .debug_abbrev  0x00000da1      0x283 lib_generic/zlib.o
 .debug_abbrev  0x00001024      0x1da lib_generic/libgeneric.a(vsprintf.o)
 .debug_abbrev  0x000011fe       0x42 lib_generic/libgeneric.a(ctype.o)
 .debug_abbrev  0x00001240      0x172 lib_generic/libgeneric.a(string.o)
 .debug_abbrev  0x000013b2      0x293 board/mpc8548pc/libmpc8548pc.a(mpc8548pc.o)
 .debug_abbrev  0x00001645      0x239 lib_ppc/libppc.a(board.o)
 .debug_abbrev  0x0000187e       0xa9 lib_ppc/libppc.a(time.o)
 .debug_abbrev  0x00001927      0x2c6 net/libnet.a(net.o)
 .debug_abbrev  0x00001bed      0x17e net/libnet.a(tftp.o)
 .debug_abbrev  0x00001d6b      0x261 net/libnet.a(bootp.o)
 .debug_abbrev  0x00001fcc      0x115 net/libnet.a(rarp.o)
 .debug_abbrev  0x000020e1      0x1e3 net/libnet.a(eth.o)
 .debug_abbrev  0x000022c4      0x2da net/libnet.a(nfs.o)
 .debug_abbrev  0x0000259e      0x239 drivers/libdrivers.a(cfi_flash.o)
 .debug_abbrev  0x000027d7      0x1e5 drivers/libdrivers.a(pci.o)
 .debug_abbrev  0x000029bc      0x213 drivers/libdrivers.a(pci_auto.o)
 .debug_abbrev  0x00002bcf      0x194 drivers/libdrivers.a(pci_indirect.o)
 .debug_abbrev  0x00002d63      0x143 drivers/libdrivers.a(serial.o)
 .debug_abbrev  0x00002ea6      0x2f2 drivers/libdrivers.a(tsec.o)
 .debug_abbrev  0x00003198       0xca drivers/libdrivers.a(ns16550.o)
 .debug_abbrev  0x00003262      0x1fb common/libcommon.a(main.o)
 .debug_abbrev  0x0000345d      0x106 common/libcommon.a(cmd_autoscript.o)
 .debug_abbrev  0x00003563      0x112 common/libcommon.a(cmd_bdinfo.o)
 .debug_abbrev  0x00003675       0xd6 common/libcommon.a(cmd_boot.o)
 .debug_abbrev  0x0000374b      0x291 common/libcommon.a(cmd_bootm.o)
 .debug_abbrev  0x000039dc      0x132 common/libcommon.a(cmd_console.o)
 .debug_abbrev  0x00003b0e      0x1a4 common/libcommon.a(cmd_flash.o)
 .debug_abbrev  0x00003cb2      0x17e common/libcommon.a(cmd_i2c.o)
 .debug_abbrev  0x00003e30      0x17f common/libcommon.a(cmd_itest.o)
 .debug_abbrev  0x00003faf      0x2d6 common/libcommon.a(cmd_load.o)
 .debug_abbrev  0x00004285      0x1c0 common/libcommon.a(cmd_mem.o)
 .debug_abbrev  0x00004445      0x213 common/libcommon.a(cmd_mii.o)
 .debug_abbrev  0x00004658       0xc7 common/libcommon.a(cmd_misc.o)
 .debug_abbrev  0x0000471f      0x17b common/libcommon.a(cmd_net.o)
 .debug_abbrev  0x0000489a      0x1d0 common/libcommon.a(cmd_nvedit.o)
 .debug_abbrev  0x00004a6a      0x25c common/libcommon.a(cmd_pci.o)
 .debug_abbrev  0x00004cc6      0x182 common/libcommon.a(command.o)
 .debug_abbrev  0x00004e48      0x220 common/libcommon.a(console.o)
 .debug_abbrev  0x00005068      0x161 common/libcommon.a(devices.o)
 .debug_abbrev  0x000051c9      0x153 common/libcommon.a(env_common.o)
 .debug_abbrev  0x0000531c      0x16b common/libcommon.a(env_flash.o)
 .debug_abbrev  0x00005487       0xdd common/libcommon.a(exports.o)
 .debug_abbrev  0x00005564      0x109 common/libcommon.a(flash.o)
 .debug_abbrev  0x0000566d      0x2e4 common/libcommon.a(hush.o)
 .debug_abbrev  0x00005951      0x18e common/libcommon.a(lists.o)
 .debug_abbrev  0x00005adf      0x1ae common/libcommon.a(miiphyutil.o)
 .debug_abbrev  0x00005c8d       0xac common/libcommon.a(s_record.o)
 .debug_abbrev  0x00005d39       0xc3 lib_generic/libgeneric.a(display_options.o)
 .debug_abbrev  0x00005dfc      0x1ce cpu/mpc85xx/libmpc85xx.a(i2c.o)
 .debug_abbrev  0x00005fca       0x6a lib_ppc/libppc.a(cache.o)

.debug_info     0x00000000    0x3a058
 .debug_info    0x00000000      0x5da cpu/mpc85xx/traps.o
 .debug_info    0x000005da     0x56e8 cpu/mpc85xx/interrupts.o
 .debug_info    0x00005cc2     0x55e5 cpu/mpc85xx/cpu_init.o
 .debug_info    0x0000b2a7     0x5764 cpu/mpc85xx/cpu.o
 .debug_info    0x00010a0b     0x564d cpu/mpc85xx/speed.o
 .debug_info    0x00016058     0x57d4 cpu/mpc85xx/pci.o
 .debug_info    0x0001b82c      0xbd5 common/dlmalloc.o
 .debug_info    0x0001c401      0x12a lib_generic/crc32.o
 .debug_info    0x0001c52b      0x1ac lib_ppc/extable.o
 .debug_info    0x0001c6d7     0x16a6 lib_generic/zlib.o
 .debug_info    0x0001dd7d      0x46b lib_generic/libgeneric.a(vsprintf.o)
 .debug_info    0x0001e1e8       0x56 lib_generic/libgeneric.a(ctype.o)
 .debug_info    0x0001e23e      0x54f lib_generic/libgeneric.a(string.o)
 .debug_info    0x0001e78d     0x6932 board/mpc8548pc/libmpc8548pc.a(mpc8548pc.o)
 .debug_info    0x000250bf      0x6f9 lib_ppc/libppc.a(board.o)
 .debug_info    0x000257b8      0x136 lib_ppc/libppc.a(time.o)
 .debug_info    0x000258ee     0x1459 net/libnet.a(net.o)
 .debug_info    0x00026d47      0x3b1 net/libnet.a(tftp.o)
 .debug_info    0x000270f8      0x846 net/libnet.a(bootp.o)
 .debug_info    0x0002793e      0x243 net/libnet.a(rarp.o)
 .debug_info    0x00027b81      0x63e net/libnet.a(eth.o)
 .debug_info    0x000281bf      0xc42 net/libnet.a(nfs.o)
 .debug_info    0x00028e01      0xec7 drivers/libdrivers.a(cfi_flash.o)
 .debug_info    0x00029cc8      0xf31 drivers/libdrivers.a(pci.o)
 .debug_info    0x0002abf9      0x767 drivers/libdrivers.a(pci_auto.o)
 .debug_info    0x0002b360      0x8ac drivers/libdrivers.a(pci_indirect.o)
 .debug_info    0x0002bc0c      0x554 drivers/libdrivers.a(serial.o)
 .debug_info    0x0002c160     0x1d7e drivers/libdrivers.a(tsec.o)
 .debug_info    0x0002dede      0x1b0 drivers/libdrivers.a(ns16550.o)
 .debug_info    0x0002e08e      0x5e4 common/libcommon.a(main.o)
 .debug_info    0x0002e672      0x34e common/libcommon.a(cmd_autoscript.o)
 .debug_info    0x0002e9c0      0x43a common/libcommon.a(cmd_bdinfo.o)
 .debug_info    0x0002edfa      0x1c8 common/libcommon.a(cmd_boot.o)
 .debug_info    0x0002efc2     0x11b7 common/libcommon.a(cmd_bootm.o)
 .debug_info    0x00030179      0x379 common/libcommon.a(cmd_console.o)
 .debug_info    0x000304f2      0x83c common/libcommon.a(cmd_flash.o)
 .debug_info    0x00030d2e      0x782 common/libcommon.a(cmd_i2c.o)
 .debug_info    0x000314b0      0x42c common/libcommon.a(cmd_itest.o)
 .debug_info    0x000318dc      0xc77 common/libcommon.a(cmd_load.o)
 .debug_info    0x00032553      0xa10 common/libcommon.a(cmd_mem.o)
 .debug_info    0x00032f63      0x746 common/libcommon.a(cmd_mii.o)
 .debug_info    0x000336a9      0x1aa common/libcommon.a(cmd_misc.o)
 .debug_info    0x00033853      0x533 common/libcommon.a(cmd_net.o)
 .debug_info    0x00033d86      0x85f common/libcommon.a(cmd_nvedit.o)
 .debug_info    0x000345e5      0x6ce common/libcommon.a(cmd_pci.o)
 .debug_info    0x00034cb3      0x521 common/libcommon.a(command.o)
 .debug_info    0x000351d4      0x9f6 common/libcommon.a(console.o)
 .debug_info    0x00035bca      0x520 common/libcommon.a(devices.o)
 .debug_info    0x000360ea      0x40a common/libcommon.a(env_common.o)
 .debug_info    0x000364f4      0x429 common/libcommon.a(env_flash.o)
 .debug_info    0x0003691d      0x2cd common/libcommon.a(exports.o)
 .debug_info    0x00036bea      0x37b common/libcommon.a(flash.o)
 .debug_info    0x00036f65     0x176d common/libcommon.a(hush.o)
 .debug_info    0x000386d2      0x4df common/libcommon.a(lists.o)
 .debug_info    0x00038bb1      0x57e common/libcommon.a(miiphyutil.o)
 .debug_info    0x0003912f      0x179 common/libcommon.a(s_record.o)
 .debug_info    0x000392a8      0x120 lib_generic/libgeneric.a(display_options.o)
 .debug_info    0x000393c8      0xbc3 cpu/mpc85xx/libmpc85xx.a(i2c.o)
 .debug_info    0x00039f8b       0xcd lib_ppc/libppc.a(cache.o)

.debug_line     0x00000000     0x6ca7
 .debug_line    0x00000000      0x14c cpu/mpc85xx/traps.o
 .debug_line    0x0000014c      0x14d cpu/mpc85xx/interrupts.o
 .debug_line    0x00000299      0x119 cpu/mpc85xx/cpu_init.o
 .debug_line    0x000003b2      0x174 cpu/mpc85xx/cpu.o
 .debug_line    0x00000526      0x130 cpu/mpc85xx/speed.o
 .debug_line    0x00000656      0x189 cpu/mpc85xx/pci.o
 .debug_line    0x000007df      0x3b4 common/dlmalloc.o
 .debug_line    0x00000b93       0x7c lib_generic/crc32.o
 .debug_line    0x00000c0f       0x53 lib_ppc/extable.o
 .debug_line    0x00000c62      0x61a lib_generic/zlib.o
 .debug_line    0x0000127c      0x1ea lib_generic/libgeneric.a(vsprintf.o)
 .debug_line    0x00001466       0x25 lib_generic/libgeneric.a(ctype.o)
 .debug_line    0x0000148b      0x188 lib_generic/libgeneric.a(string.o)
 .debug_line    0x00001613      0x2c2 board/mpc8548pc/libmpc8548pc.a(mpc8548pc.o)
 .debug_line    0x000018d5      0x287 lib_ppc/libppc.a(board.o)
 .debug_line    0x00001b5c       0x8f lib_ppc/libppc.a(time.o)
 .debug_line    0x00001beb      0x4ef net/libnet.a(net.o)
 .debug_line    0x000020da      0x1a3 net/libnet.a(tftp.o)
 .debug_line    0x0000227d      0x28b net/libnet.a(bootp.o)
 .debug_line    0x00002508       0xd7 net/libnet.a(rarp.o)
 .debug_line    0x000025df      0x166 net/libnet.a(eth.o)
 .debug_line    0x00002745      0x2be net/libnet.a(nfs.o)
 .debug_line    0x00002a03      0x3df drivers/libdrivers.a(cfi_flash.o)
 .debug_line    0x00002de2      0x1b6 drivers/libdrivers.a(pci.o)
 .debug_line    0x00002f98      0x174 drivers/libdrivers.a(pci_auto.o)
 .debug_line    0x0000310c      0x142 drivers/libdrivers.a(pci_indirect.o)
 .debug_line    0x0000324e      0x101 drivers/libdrivers.a(serial.o)
 .debug_line    0x0000334f      0x3c7 drivers/libdrivers.a(tsec.o)
 .debug_line    0x00003716       0x8f drivers/libdrivers.a(ns16550.o)
 .debug_line    0x000037a5      0x1d3 common/libcommon.a(main.o)
 .debug_line    0x00003978      0x12f common/libcommon.a(cmd_autoscript.o)
 .debug_line    0x00003aa7      0x13b common/libcommon.a(cmd_bdinfo.o)
 .debug_line    0x00003be2       0xc3 common/libcommon.a(cmd_boot.o)
 .debug_line    0x00003ca5      0x35d common/libcommon.a(cmd_bootm.o)
 .debug_line    0x00004002       0xab common/libcommon.a(cmd_console.o)
 .debug_line    0x000040ad      0x259 common/libcommon.a(cmd_flash.o)
 .debug_line    0x00004306      0x22a common/libcommon.a(cmd_i2c.o)
 .debug_line    0x00004530      0x108 common/libcommon.a(cmd_itest.o)
 .debug_line    0x00004638      0x330 common/libcommon.a(cmd_load.o)
 .debug_line    0x00004968      0x298 common/libcommon.a(cmd_mem.o)
 .debug_line    0x00004c00      0x1b7 common/libcommon.a(cmd_mii.o)
 .debug_line    0x00004db7       0xba common/libcommon.a(cmd_misc.o)
 .debug_line    0x00004e71      0x12d common/libcommon.a(cmd_net.o)
 .debug_line    0x00004f9e      0x230 common/libcommon.a(cmd_nvedit.o)
 .debug_line    0x000051ce      0x246 common/libcommon.a(cmd_pci.o)
 .debug_line    0x00005414      0x16b common/libcommon.a(command.o)
 .debug_line    0x0000557f      0x2c7 common/libcommon.a(console.o)
 .debug_line    0x00005846      0x138 common/libcommon.a(devices.o)
 .debug_line    0x0000597e      0x103 common/libcommon.a(env_common.o)
 .debug_line    0x00005a81      0x158 common/libcommon.a(env_flash.o)
 .debug_line    0x00005bd9       0xa1 common/libcommon.a(exports.o)
 .debug_line    0x00005c7a      0x13d common/libcommon.a(flash.o)
 .debug_line    0x00005db7      0x62f common/libcommon.a(hush.o)
 .debug_line    0x000063e6      0x118 common/libcommon.a(lists.o)
 .debug_line    0x000064fe      0x222 common/libcommon.a(miiphyutil.o)
 .debug_line    0x00006720       0xfb common/libcommon.a(s_record.o)
 .debug_line    0x0000681b       0x95 lib_generic/libgeneric.a(display_options.o)
 .debug_line    0x000068b0      0x37e cpu/mpc85xx/libmpc85xx.a(i2c.o)
 .debug_line    0x00006c2e       0x79 lib_ppc/libppc.a(cache.o)

.debug_frame    0x00000000     0x3d0c
 .debug_frame   0x00000000      0x158 cpu/mpc85xx/traps.o
 .debug_frame   0x00000158       0xec cpu/mpc85xx/interrupts.o
 .debug_frame   0x00000244       0x4c cpu/mpc85xx/cpu_init.o
 .debug_frame   0x00000290       0xac cpu/mpc85xx/cpu.o
 .debug_frame   0x0000033c       0x64 cpu/mpc85xx/speed.o
 .debug_frame   0x000003a0       0x34 cpu/mpc85xx/pci.o
 .debug_frame   0x000003d4      0x188 common/dlmalloc.o
 .debug_frame   0x0000055c       0x2c lib_generic/crc32.o
 .debug_frame   0x00000588       0x2c lib_ppc/extable.o
 .debug_frame   0x000005b4      0x240 lib_generic/zlib.o
 .debug_frame   0x000007f4       0xd4 lib_generic/libgeneric.a(vsprintf.o)
 .debug_frame   0x000008c8      0x16c lib_generic/libgeneric.a(string.o)
 .debug_frame   0x00000a34      0x190 board/mpc8548pc/libmpc8548pc.a(mpc8548pc.o)
 .debug_frame   0x00000bc4      0x110 lib_ppc/libppc.a(board.o)
 .debug_frame   0x00000cd4       0x7c lib_ppc/libppc.a(time.o)
 .debug_frame   0x00000d50      0x33c net/libnet.a(net.o)
 .debug_frame   0x0000108c       0x98 net/libnet.a(tftp.o)
 .debug_frame   0x00001124       0x9c net/libnet.a(bootp.o)
 .debug_frame   0x000011c0       0x64 net/libnet.a(rarp.o)
 .debug_frame   0x00001224      0x1b4 net/libnet.a(eth.o)
 .debug_frame   0x000013d8      0x164 net/libnet.a(nfs.o)
 .debug_frame   0x0000153c      0x258 drivers/libdrivers.a(cfi_flash.o)
 .debug_frame   0x00001794      0x38c drivers/libdrivers.a(pci.o)
 .debug_frame   0x00001b20       0xc0 drivers/libdrivers.a(pci_auto.o)
 .debug_frame   0x00001be0       0xa4 drivers/libdrivers.a(pci_indirect.o)
 .debug_frame   0x00001c84      0x18c drivers/libdrivers.a(serial.o)
 .debug_frame   0x00001e10      0x258 drivers/libdrivers.a(tsec.o)
 .debug_frame   0x00002068       0x74 drivers/libdrivers.a(ns16550.o)
 .debug_frame   0x000020dc       0xd8 common/libcommon.a(main.o)
 .debug_frame   0x000021b4       0x54 common/libcommon.a(cmd_autoscript.o)
 .debug_frame   0x00002208       0x6c common/libcommon.a(cmd_bdinfo.o)
 .debug_frame   0x00002274       0x34 common/libcommon.a(cmd_boot.o)
 .debug_frame   0x000022a8      0x15c common/libcommon.a(cmd_bootm.o)
 .debug_frame   0x00002404       0x34 common/libcommon.a(cmd_console.o)
 .debug_frame   0x00002438      0x138 common/libcommon.a(cmd_flash.o)
 .debug_frame   0x00002570      0x128 common/libcommon.a(cmd_i2c.o)
 .debug_frame   0x00002698       0x8c common/libcommon.a(cmd_itest.o)
 .debug_frame   0x00002724      0x1fc common/libcommon.a(cmd_load.o)
 .debug_frame   0x00002920      0x1b8 common/libcommon.a(cmd_mem.o)
 .debug_frame   0x00002ad8       0x8c common/libcommon.a(cmd_mii.o)
 .debug_frame   0x00002b64       0x34 common/libcommon.a(cmd_misc.o)
 .debug_frame   0x00002b98       0xa8 common/libcommon.a(cmd_net.o)
 .debug_frame   0x00002c40      0x130 common/libcommon.a(cmd_nvedit.o)
 .debug_frame   0x00002d70      0x10c common/libcommon.a(cmd_pci.o)
 .debug_frame   0x00002e7c       0xf0 common/libcommon.a(command.o)
 .debug_frame   0x00002f6c      0x26c common/libcommon.a(console.o)
 .debug_frame   0x000031d8       0x68 common/libcommon.a(devices.o)
 .debug_frame   0x00003240       0xa0 common/libcommon.a(env_common.o)
 .debug_frame   0x000032e0       0x88 common/libcommon.a(env_flash.o)
 .debug_frame   0x00003368       0x54 common/libcommon.a(exports.o)
 .debug_frame   0x000033bc       0x88 common/libcommon.a(flash.o)
 .debug_frame   0x00003444      0x404 common/libcommon.a(hush.o)
 .debug_frame   0x00003848      0x17c common/libcommon.a(lists.o)
 .debug_frame   0x000039c4      0x198 common/libcommon.a(miiphyutil.o)
 .debug_frame   0x00003b5c       0x70 common/libcommon.a(s_record.o)
 .debug_frame   0x00003bcc       0x50 lib_generic/libgeneric.a(display_options.o)
 .debug_frame   0x00003c1c       0xcc cpu/mpc85xx/libmpc85xx.a(i2c.o)
 .debug_frame   0x00003ce8       0x24 lib_ppc/libppc.a(cache.o)

.debug_pubnames
                0x00000000     0x287a
 .debug_pubnames
                0x00000000       0xf0 cpu/mpc85xx/traps.o
 .debug_pubnames
                0x000000f0       0xe3 cpu/mpc85xx/interrupts.o
 .debug_pubnames
                0x000001d3       0x30 cpu/mpc85xx/cpu_init.o
 .debug_pubnames
                0x00000203       0x62 cpu/mpc85xx/cpu.o
 .debug_pubnames
                0x00000265       0x43 cpu/mpc85xx/speed.o
 .debug_pubnames
                0x000002a8       0x27 cpu/mpc85xx/pci.o
 .debug_pubnames
                0x000002cf       0xb3 common/dlmalloc.o
 .debug_pubnames
                0x00000382       0x1c lib_generic/crc32.o
 .debug_pubnames
                0x0000039e       0x40 lib_ppc/extable.o
 .debug_pubnames
                0x000003de       0xab lib_generic/zlib.o
 .debug_pubnames
                0x00000489       0x5a lib_generic/libgeneric.a(vsprintf.o)
 .debug_pubnames
                0x000004e3       0x1d lib_generic/libgeneric.a(ctype.o)
 .debug_pubnames
                0x00000500       0xc3 lib_generic/libgeneric.a(string.o)
 .debug_pubnames
                0x000005c3       0xea board/mpc8548pc/libmpc8548pc.a(mpc8548pc.o)
 .debug_pubnames
                0x000006ad       0x79 lib_ppc/libppc.a(board.o)
 .debug_pubnames
                0x00000726       0x4d lib_ppc/libppc.a(time.o)
 .debug_pubnames
                0x00000773      0x405 net/libnet.a(net.o)
 .debug_pubnames
                0x00000b78       0x20 net/libnet.a(tftp.o)
 .debug_pubnames
                0x00000b98       0x3c net/libnet.a(bootp.o)
 .debug_pubnames
                0x00000bd4       0x2e net/libnet.a(rarp.o)
 .debug_pubnames
                0x00000c02       0xf4 net/libnet.a(eth.o)
 .debug_pubnames
                0x00000cf6       0x1f net/libnet.a(nfs.o)
 .debug_pubnames
                0x00000d15       0xca drivers/libdrivers.a(cfi_flash.o)
 .debug_pubnames
                0x00000ddf      0x32a drivers/libdrivers.a(pci.o)
 .debug_pubnames
                0x00001109       0xaa drivers/libdrivers.a(pci_auto.o)
 .debug_pubnames
                0x000011b3       0x29 drivers/libdrivers.a(pci_indirect.o)
 .debug_pubnames
                0x000011dc       0xf4 drivers/libdrivers.a(serial.o)
 .debug_pubnames
                0x000012d0      0x222 drivers/libdrivers.a(tsec.o)
 .debug_pubnames
                0x000014f2       0x69 drivers/libdrivers.a(ns16550.o)
 .debug_pubnames
                0x0000155b       0x5b common/libcommon.a(main.o)
 .debug_pubnames
                0x000015b6       0x4c common/libcommon.a(cmd_autoscript.o)
 .debug_pubnames
                0x00001602       0x38 common/libcommon.a(cmd_bdinfo.o)
 .debug_pubnames
                0x0000163a       0x47 common/libcommon.a(cmd_boot.o)
 .debug_pubnames
                0x00001681       0xe4 common/libcommon.a(cmd_bootm.o)
 .debug_pubnames
                0x00001765       0x3a common/libcommon.a(cmd_console.o)
 .debug_pubnames
                0x0000179f       0xb2 common/libcommon.a(cmd_flash.o)
 .debug_pubnames
                0x00001851      0x115 common/libcommon.a(cmd_i2c.o)
 .debug_pubnames
                0x00001966       0x53 common/libcommon.a(cmd_itest.o)
 .debug_pubnames
                0x000019b9      0x1b2 common/libcommon.a(cmd_load.o)
 .debug_pubnames
                0x00001b6b      0x1e7 common/libcommon.a(cmd_mem.o)
 .debug_pubnames
                0x00001d52      0x13e common/libcommon.a(cmd_mii.o)
 .debug_pubnames
                0x00001e90       0x36 common/libcommon.a(cmd_misc.o)
 .debug_pubnames
                0x00001ec6       0xc6 common/libcommon.a(cmd_net.o)
 .debug_pubnames
                0x00001f8c       0xd1 common/libcommon.a(cmd_nvedit.o)
 .debug_pubnames
                0x0000205d       0x80 common/libcommon.a(cmd_pci.o)
 .debug_pubnames
                0x000020dd       0xee common/libcommon.a(command.o)
 .debug_pubnames
                0x000021cb      0x10e common/libcommon.a(console.o)
 .debug_pubnames
                0x000022d9       0x76 common/libcommon.a(devices.o)
 .debug_pubnames
                0x0000234f       0x88 common/libcommon.a(env_common.o)
 .debug_pubnames
                0x000023d7       0x75 common/libcommon.a(env_flash.o)
 .debug_pubnames
                0x0000244c       0x35 common/libcommon.a(exports.o)
 .debug_pubnames
                0x00002481       0x53 common/libcommon.a(flash.o)
 .debug_pubnames
                0x000024d4       0xc8 common/libcommon.a(hush.o)
 .debug_pubnames
                0x0000259c      0x116 common/libcommon.a(lists.o)
 .debug_pubnames
                0x000026b2       0xe4 common/libcommon.a(miiphyutil.o)
 .debug_pubnames
                0x00002796       0x22 common/libcommon.a(s_record.o)
 .debug_pubnames
                0x000027b8       0x35 lib_generic/libgeneric.a(display_options.o)
 .debug_pubnames
                0x000027ed       0x6b cpu/mpc85xx/libmpc85xx.a(i2c.o)
 .debug_pubnames
                0x00002858       0x22 lib_ppc/libppc.a(cache.o)

.debug_aranges  0x00000000      0x740
 .debug_aranges
                0x00000000       0x20 cpu/mpc85xx/traps.o
 .debug_aranges
                0x00000020       0x20 cpu/mpc85xx/interrupts.o
 .debug_aranges
                0x00000040       0x20 cpu/mpc85xx/cpu_init.o
 .debug_aranges
                0x00000060       0x20 cpu/mpc85xx/cpu.o
 .debug_aranges
                0x00000080       0x20 cpu/mpc85xx/speed.o
 .debug_aranges
                0x000000a0       0x20 cpu/mpc85xx/pci.o
 .debug_aranges
                0x000000c0       0x20 common/dlmalloc.o
 .debug_aranges
                0x000000e0       0x20 lib_generic/crc32.o
 .debug_aranges
                0x00000100       0x20 lib_ppc/extable.o
 .debug_aranges
                0x00000120       0x20 lib_generic/zlib.o
 .debug_aranges
                0x00000140       0x20 lib_generic/libgeneric.a(vsprintf.o)
 .debug_aranges
                0x00000160       0x20 lib_generic/libgeneric.a(string.o)
 .debug_aranges
                0x00000180       0x20 board/mpc8548pc/libmpc8548pc.a(mpc8548pc.o)
 .debug_aranges
                0x000001a0       0x20 lib_ppc/libppc.a(board.o)
 .debug_aranges
                0x000001c0       0x20 lib_ppc/libppc.a(time.o)
 .debug_aranges
                0x000001e0       0x20 net/libnet.a(net.o)
 .debug_aranges
                0x00000200       0x20 net/libnet.a(tftp.o)
 .debug_aranges
                0x00000220       0x20 net/libnet.a(bootp.o)
 .debug_aranges
                0x00000240       0x20 net/libnet.a(rarp.o)
 .debug_aranges
                0x00000260       0x20 net/libnet.a(eth.o)
 .debug_aranges
                0x00000280       0x20 net/libnet.a(nfs.o)
 .debug_aranges
                0x000002a0       0x20 drivers/libdrivers.a(cfi_flash.o)
 .debug_aranges
                0x000002c0       0x20 drivers/libdrivers.a(pci.o)
 .debug_aranges
                0x000002e0       0x20 drivers/libdrivers.a(pci_auto.o)
 .debug_aranges
                0x00000300       0x20 drivers/libdrivers.a(pci_indirect.o)
 .debug_aranges
                0x00000320       0x20 drivers/libdrivers.a(serial.o)
 .debug_aranges
                0x00000340       0x20 drivers/libdrivers.a(tsec.o)
 .debug_aranges
                0x00000360       0x20 drivers/libdrivers.a(ns16550.o)
 .debug_aranges
                0x00000380       0x20 common/libcommon.a(main.o)
 .debug_aranges
                0x000003a0       0x20 common/libcommon.a(cmd_autoscript.o)
 .debug_aranges
                0x000003c0       0x20 common/libcommon.a(cmd_bdinfo.o)
 .debug_aranges
                0x000003e0       0x20 common/libcommon.a(cmd_boot.o)
 .debug_aranges
                0x00000400       0x20 common/libcommon.a(cmd_bootm.o)
 .debug_aranges
                0x00000420       0x20 common/libcommon.a(cmd_console.o)
 .debug_aranges
                0x00000440       0x20 common/libcommon.a(cmd_flash.o)
 .debug_aranges
                0x00000460       0x20 common/libcommon.a(cmd_i2c.o)
 .debug_aranges
                0x00000480       0x20 common/libcommon.a(cmd_itest.o)
 .debug_aranges
                0x000004a0       0x20 common/libcommon.a(cmd_load.o)
 .debug_aranges
                0x000004c0       0x20 common/libcommon.a(cmd_mem.o)
 .debug_aranges
                0x000004e0       0x20 common/libcommon.a(cmd_mii.o)
 .debug_aranges
                0x00000500       0x20 common/libcommon.a(cmd_misc.o)
 .debug_aranges
                0x00000520       0x20 common/libcommon.a(cmd_net.o)
 .debug_aranges
                0x00000540       0x20 common/libcommon.a(cmd_nvedit.o)
 .debug_aranges
                0x00000560       0x20 common/libcommon.a(cmd_pci.o)
 .debug_aranges
                0x00000580       0x20 common/libcommon.a(command.o)
 .debug_aranges
                0x000005a0       0x20 common/libcommon.a(console.o)
 .debug_aranges
                0x000005c0       0x20 common/libcommon.a(devices.o)
 .debug_aranges
                0x000005e0       0x20 common/libcommon.a(env_common.o)
 .debug_aranges
                0x00000600       0x20 common/libcommon.a(env_flash.o)
 .debug_aranges
                0x00000620       0x20 common/libcommon.a(exports.o)
 .debug_aranges
                0x00000640       0x20 common/libcommon.a(flash.o)
 .debug_aranges
                0x00000660       0x20 common/libcommon.a(hush.o)
 .debug_aranges
                0x00000680       0x20 common/libcommon.a(lists.o)
 .debug_aranges
                0x000006a0       0x20 common/libcommon.a(miiphyutil.o)
 .debug_aranges
                0x000006c0       0x20 common/libcommon.a(s_record.o)
 .debug_aranges
                0x000006e0       0x20 lib_generic/libgeneric.a(display_options.o)
 .debug_aranges
                0x00000700       0x20 cpu/mpc85xx/libmpc85xx.a(i2c.o)
 .debug_aranges
                0x00000720       0x20 lib_ppc/libppc.a(cache.o)

.debug_str      0x00000000     0x6568
 .debug_str     0x00000000      0x2f3 cpu/mpc85xx/traps.o
                                0x353 (size before relaxing)
 .debug_str     0x000002f3     0x1a95 cpu/mpc85xx/interrupts.o
                               0x1c4f (size before relaxing)
 .debug_str     0x00001d88       0x42 cpu/mpc85xx/cpu_init.o
                               0x1cd2 (size before relaxing)
 .debug_str     0x00001dca       0xce cpu/mpc85xx/cpu.o
                               0x1d15 (size before relaxing)
 .debug_str     0x00001e98       0x51 cpu/mpc85xx/speed.o
                               0x1d20 (size before relaxing)
 .debug_str     0x00001ee9      0x111 cpu/mpc85xx/pci.o
                               0x1c92 (size before relaxing)
 .debug_str     0x00001ffa      0x2e3 common/dlmalloc.o
                                0x54a (size before relaxing)
 .debug_str     0x000022dd       0x5d lib_generic/crc32.o
                                0x10e (size before relaxing)
 .debug_str     0x0000233a       0xb0 lib_ppc/extable.o
                                0x177 (size before relaxing)
 .debug_str     0x000023ea      0x46d lib_generic/zlib.o
                                0x5c8 (size before relaxing)
 .debug_str     0x00002857       0xca lib_generic/libgeneric.a(vsprintf.o)
                                0x1ed (size before relaxing)
 .debug_str     0x00002921        0x8 lib_generic/libgeneric.a(ctype.o)
                                 0x7a (size before relaxing)
 .debug_str     0x00002929       0x8f lib_generic/libgeneric.a(string.o)
                                0x1ad (size before relaxing)
 .debug_str     0x000029b8      0x337 board/mpc8548pc/libmpc8548pc.a(mpc8548pc.o)
                               0x212c (size before relaxing)
 .debug_str     0x00002cef      0x167 lib_ppc/libppc.a(board.o)
                                0x41a (size before relaxing)
 .debug_str     0x00002e56       0x32 lib_ppc/libppc.a(time.o)
                                0x11e (size before relaxing)
 .debug_str     0x00002e88      0x5dd net/libnet.a(net.o)
                                0x870 (size before relaxing)
 .debug_str     0x00003465       0xe4 net/libnet.a(tftp.o)
                                0x27c (size before relaxing)
 .debug_str     0x00003549      0x176 net/libnet.a(bootp.o)
                                0x36a (size before relaxing)
 .debug_str     0x000036bf       0x4c net/libnet.a(rarp.o)
                                0x1a8 (size before relaxing)
 .debug_str     0x0000370b      0x12f net/libnet.a(eth.o)
                                0x353 (size before relaxing)
 .debug_str     0x0000383a      0x271 net/libnet.a(nfs.o)
                                0x467 (size before relaxing)
 .debug_str     0x00003aab      0x2cd drivers/libdrivers.a(cfi_flash.o)
                                0x417 (size before relaxing)
 .debug_str     0x00003d78      0x33e drivers/libdrivers.a(pci.o)
                                0x5a1 (size before relaxing)
 .debug_str     0x000040b6       0xf0 drivers/libdrivers.a(pci_auto.o)
                                0x353 (size before relaxing)
 .debug_str     0x000041a6       0xfc drivers/libdrivers.a(pci_indirect.o)
                                0x333 (size before relaxing)
 .debug_str     0x000042a2       0xa3 drivers/libdrivers.a(serial.o)
                                0x328 (size before relaxing)
 .debug_str     0x00004345      0x4cc drivers/libdrivers.a(tsec.o)
                                0xbcb (size before relaxing)
 .debug_str     0x00004811       0x63 drivers/libdrivers.a(ns16550.o)
                                 0xd4 (size before relaxing)
 .debug_str     0x00004874       0xeb common/libcommon.a(main.o)
                                0x241 (size before relaxing)
 .debug_str     0x0000495f       0xbc common/libcommon.a(cmd_autoscript.o)
                                0x220 (size before relaxing)
 .debug_str     0x00004a1b       0x3f common/libcommon.a(cmd_bdinfo.o)
                                0x2c8 (size before relaxing)
 .debug_str     0x00004a5a       0x34 common/libcommon.a(cmd_boot.o)
                                0x165 (size before relaxing)
 .debug_str     0x00004a8e      0x194 common/libcommon.a(cmd_bootm.o)
                                0x6a1 (size before relaxing)
 .debug_str     0x00004c22       0xc5 common/libcommon.a(cmd_console.o)
                                0x204 (size before relaxing)
 .debug_str     0x00004ce7      0x132 common/libcommon.a(cmd_flash.o)
                                0x349 (size before relaxing)
 .debug_str     0x00004e19      0x18a common/libcommon.a(cmd_i2c.o)
                                0x312 (size before relaxing)
 .debug_str     0x00004fa3       0x80 common/libcommon.a(cmd_itest.o)
                                0x1c0 (size before relaxing)
 .debug_str     0x00005023      0x2d5 common/libcommon.a(cmd_load.o)
                                0x5d6 (size before relaxing)
 .debug_str     0x000052f8      0x1c1 common/libcommon.a(cmd_mem.o)
                                0x399 (size before relaxing)
 .debug_str     0x000054b9      0x1b0 common/libcommon.a(cmd_mii.o)
                                0x34f (size before relaxing)
 .debug_str     0x00005669       0x27 common/libcommon.a(cmd_misc.o)
                                0x159 (size before relaxing)
 .debug_str     0x00005690       0xc3 common/libcommon.a(cmd_net.o)
                                0x2bf (size before relaxing)
 .debug_str     0x00005753       0xd5 common/libcommon.a(cmd_nvedit.o)
                                0x3a3 (size before relaxing)
 .debug_str     0x00005828       0xfb common/libcommon.a(cmd_pci.o)
                                0x2bd (size before relaxing)
 .debug_str     0x00005923      0x103 common/libcommon.a(command.o)
                                0x25f (size before relaxing)
 .debug_str     0x00005a26       0xd7 common/libcommon.a(console.o)
                                0x468 (size before relaxing)
 .debug_str     0x00005afd       0x56 common/libcommon.a(devices.o)
                                0x348 (size before relaxing)
 .debug_str     0x00005b53       0x8c common/libcommon.a(env_common.o)
                                0x2db (size before relaxing)
 .debug_str     0x00005bdf       0x6c common/libcommon.a(env_flash.o)
                                0x309 (size before relaxing)
 .debug_str     0x00005c4b       0x25 common/libcommon.a(exports.o)
                                0x25c (size before relaxing)
 .debug_str     0x00005c70       0x46 common/libcommon.a(flash.o)
                                0x204 (size before relaxing)
 .debug_str     0x00005cb6      0x4d7 common/libcommon.a(hush.o)
                                0x832 (size before relaxing)
 .debug_str     0x0000618d      0x1dc common/libcommon.a(lists.o)
                                0x328 (size before relaxing)
 .debug_str     0x00006369      0x105 common/libcommon.a(miiphyutil.o)
                                0x248 (size before relaxing)
 .debug_str     0x0000646e       0x3a common/libcommon.a(s_record.o)
                                0x12a (size before relaxing)
 .debug_str     0x000064a8       0x2d lib_generic/libgeneric.a(display_options.o)
                                0x120 (size before relaxing)
 .debug_str     0x000064d5       0x7f cpu/mpc85xx/libmpc85xx.a(i2c.o)
                                0x1c3 (size before relaxing)
 .debug_str     0x00006554       0x14 lib_ppc/libppc.a(cache.o)
                                0x10d (size before relaxing)

.note.GNU-stack
                0x00000000        0x0

.comment        0x00000000      0x938
 .comment       0x00000000       0x28 cpu/mpc85xx/traps.o
 .comment       0x00000028       0x28 cpu/mpc85xx/interrupts.o
 .comment       0x00000050       0x28 cpu/mpc85xx/cpu_init.o
 .comment       0x00000078       0x28 cpu/mpc85xx/cpu.o
 .comment       0x000000a0       0x28 cpu/mpc85xx/speed.o
 .comment       0x000000c8       0x28 cpu/mpc85xx/pci.o
 .comment       0x000000f0       0x28 common/dlmalloc.o
 .comment       0x00000118       0x28 lib_generic/crc32.o
 .comment       0x00000140       0x28 lib_ppc/extable.o
 .comment       0x00000168       0x28 lib_generic/zlib.o
 .comment       0x00000190       0x28 lib_generic/libgeneric.a(vsprintf.o)
 .comment       0x000001b8       0x28 lib_generic/libgeneric.a(ctype.o)
 .comment       0x000001e0       0x28 lib_generic/libgeneric.a(string.o)
 .comment       0x00000208       0x28 board/mpc8548pc/libmpc8548pc.a(mpc8548pc.o)
 .comment       0x00000230       0x28 lib_ppc/libppc.a(board.o)
 .comment       0x00000258       0x28 lib_ppc/libppc.a(time.o)
 .comment       0x00000280       0x28 net/libnet.a(net.o)
 .comment       0x000002a8       0x28 net/libnet.a(tftp.o)
 .comment       0x000002d0       0x28 net/libnet.a(bootp.o)
 .comment       0x000002f8       0x28 net/libnet.a(rarp.o)
 .comment       0x00000320       0x28 net/libnet.a(eth.o)
 .comment       0x00000348       0x28 net/libnet.a(nfs.o)
 .comment       0x00000370       0x28 drivers/libdrivers.a(cfi_flash.o)
 .comment       0x00000398       0x28 drivers/libdrivers.a(pci.o)
 .comment       0x000003c0       0x28 drivers/libdrivers.a(pci_auto.o)
 .comment       0x000003e8       0x28 drivers/libdrivers.a(pci_indirect.o)
 .comment       0x00000410       0x28 drivers/libdrivers.a(serial.o)
 .comment       0x00000438       0x28 drivers/libdrivers.a(tsec.o)
 .comment       0x00000460       0x28 drivers/libdrivers.a(ns16550.o)
 .comment       0x00000488       0x28 common/libcommon.a(main.o)
 .comment       0x000004b0       0x28 common/libcommon.a(cmd_autoscript.o)
 .comment       0x000004d8       0x28 common/libcommon.a(cmd_bdinfo.o)
 .comment       0x00000500       0x28 common/libcommon.a(cmd_boot.o)
 .comment       0x00000528       0x28 common/libcommon.a(cmd_bootm.o)
 .comment       0x00000550       0x28 common/libcommon.a(cmd_console.o)
 .comment       0x00000578       0x28 common/libcommon.a(cmd_flash.o)
 .comment       0x000005a0       0x28 common/libcommon.a(cmd_i2c.o)
 .comment       0x000005c8       0x28 common/libcommon.a(cmd_itest.o)
 .comment       0x000005f0       0x28 common/libcommon.a(cmd_load.o)
 .comment       0x00000618       0x28 common/libcommon.a(cmd_mem.o)
 .comment       0x00000640       0x28 common/libcommon.a(cmd_mii.o)
 .comment       0x00000668       0x28 common/libcommon.a(cmd_misc.o)
 .comment       0x00000690       0x28 common/libcommon.a(cmd_net.o)
 .comment       0x000006b8       0x28 common/libcommon.a(cmd_nvedit.o)
 .comment       0x000006e0       0x28 common/libcommon.a(cmd_pci.o)
 .comment       0x00000708       0x28 common/libcommon.a(command.o)
 .comment       0x00000730       0x28 common/libcommon.a(console.o)
 .comment       0x00000758       0x28 common/libcommon.a(devices.o)
 .comment       0x00000780       0x28 common/libcommon.a(env_common.o)
 .comment       0x000007a8       0x28 common/libcommon.a(env_flash.o)
 .comment       0x000007d0       0x28 common/libcommon.a(exports.o)
 .comment       0x000007f8       0x28 common/libcommon.a(flash.o)
 .comment       0x00000820       0x28 common/libcommon.a(hush.o)
 .comment       0x00000848       0x28 common/libcommon.a(lists.o)
 .comment       0x00000870       0x28 common/libcommon.a(miiphyutil.o)
 .comment       0x00000898       0x28 common/libcommon.a(s_record.o)
 .comment       0x000008c0       0x28 lib_generic/libgeneric.a(display_options.o)
 .comment       0x000008e8       0x28 cpu/mpc85xx/libmpc85xx.a(i2c.o)
 .comment       0x00000910       0x28 lib_ppc/libppc.a(cache.o)

.debug_ranges   0x00000000      0x918
 .debug_ranges  0x00000000       0x38 common/dlmalloc.o
 .debug_ranges  0x00000038       0x18 lib_ppc/extable.o
 .debug_ranges  0x00000050      0x110 lib_generic/zlib.o
 .debug_ranges  0x00000160       0x20 lib_generic/libgeneric.a(vsprintf.o)
 .debug_ranges  0x00000180       0x20 board/mpc8548pc/libmpc8548pc.a(mpc8548pc.o)
 .debug_ranges  0x000001a0       0x70 net/libnet.a(net.o)
 .debug_ranges  0x00000210       0x20 net/libnet.a(tftp.o)
 .debug_ranges  0x00000230       0x48 net/libnet.a(bootp.o)
 .debug_ranges  0x00000278       0x30 net/libnet.a(eth.o)
 .debug_ranges  0x000002a8       0x60 net/libnet.a(nfs.o)
 .debug_ranges  0x00000308      0x110 drivers/libdrivers.a(cfi_flash.o)
 .debug_ranges  0x00000418       0x38 drivers/libdrivers.a(pci_auto.o)
 .debug_ranges  0x00000450       0x88 drivers/libdrivers.a(tsec.o)
 .debug_ranges  0x000004d8       0x60 common/libcommon.a(main.o)
 .debug_ranges  0x00000538       0x18 common/libcommon.a(cmd_console.o)
 .debug_ranges  0x00000550       0x20 common/libcommon.a(cmd_flash.o)
 .debug_ranges  0x00000570       0x18 common/libcommon.a(cmd_itest.o)
 .debug_ranges  0x00000588       0x58 common/libcommon.a(cmd_load.o)
 .debug_ranges  0x000005e0       0x30 common/libcommon.a(cmd_mem.o)
 .debug_ranges  0x00000610       0x28 common/libcommon.a(cmd_mii.o)
 .debug_ranges  0x00000638       0x48 common/libcommon.a(cmd_pci.o)
 .debug_ranges  0x00000680       0x20 common/libcommon.a(command.o)
 .debug_ranges  0x000006a0       0x48 common/libcommon.a(console.o)
 .debug_ranges  0x000006e8       0x18 common/libcommon.a(devices.o)
 .debug_ranges  0x00000700       0x70 common/libcommon.a(flash.o)
 .debug_ranges  0x00000770      0x128 common/libcommon.a(hush.o)
 .debug_ranges  0x00000898       0x80 cpu/mpc85xx/libmpc85xx.a(i2c.o)
